:10000000A2C20000D1C20000CFC20000CDC20000D9
:10001000CBC20000C9C20000C7C20000C5C20000B8
:10002000C3C20000C1C20000BFC20000BDC20000C8
:10003000BBC20000B9C20000B7C20000B5C20000D8
:10004000B3C200000C940512AFC20000ADC20000A4
:100050000C94D125A9C20000A7C200000C942A105C
:10006000A3C200000C944D0E0C94240E9DC20000FF
:100070009BC2000099C2000097C2000095C2000018
:100080000C94D81191C200008FC200008DC20000F4
:100090008BC2000089C2000087C2000085C2000038
:1000A00083C2000081C200000C94AB117DC200002D
:1000B0007BC2000079C2000077C200000C947E1160
:1000C00073C2000071C200006FC200006DC2000068
:1000D0006BC2000069C2000067C2000065C2000078
:1000E00063C200007E0C810C700C740C7A0CB80C8E
:1000F000850C890C8F0C930C970C9D0CA10CA50CF6
:10010000B80CAB0CAF0CB30C0F2C1C2C252C2E2CCC
:100110003B2C442CE02FE02FE02FE02FE02F512C40
:100120005E2C6B2CE02F782C812C8A2C972CA02C09
:10013000A92CB22CBB2CC42CE02FCD2CD62CDF2C20
:10014000E02FE02FE02FE82CF12CFA2CE02FE02F0D
:10015000032D102DE02FE02FE02F1D2D2A2D372D00
:10016000E02F442D4D2D562DE02FE02FE02F5F2D59
:10017000682D712DE02F7E2D8B2D982DE02FE02FF7
:10018000E02FA52DB22DBF2DE02FCC2DD92DE62DA2
:10019000E02FE02FE02FF32D002E0D2EE02F1A2E52
:1001A000232E2C2EE02FE02FE02FE02FE02FE02F4A
:1001B000E02FE02FE02FE02FE02FE02FE02FE02FC7
:1001C000E02FE02FE02FE02FE02FE02FE02FE02FB7
:1001D000E02F502E592E622EE02F6B2E742E7D2E86
:1001E000E02FE02FE02F862E932EA02EE02FAD2EB5
:1001F000BA2EC72EE02FE02FE02FD42EE12EEE2EC8
:10020000E02FFB2E042F0D2FE02FE02FE02F162FD5
:100210001F2F282FE02FE02FE02FE02FE02FE02FDF
:10022000E02FE02FE02FE02FE02F352E3E2E472E3F
:10023000E02FE02FE02FE02FE02FE02FE02FE02F46
:10024000E02FE02FE02FE02FE02FE02FE02FE02F36
:10025000E02FE02FE02FE02FE02FE02FE02FE02F26
:10026000E02FE02FE02FE02FE02FE02FE02FE02F16
:10027000E02FE02FE02FE02FE02FE02FE02FE02F06
:10028000E02FE02FE02FE02FE02FE02FE02FE02FF6
:10029000E02FE02FE02FE02FE02F312F3A2F472FD4
:1002A000E02F542F5D2F6A2FE02FE02FE02F772FC4
:1002B000802F8D2FE02F9A2FA32FB02FE02FE02F2C
:1002C000E02FBD2FC62FD32FAE33B333B833C23395
:1002D000CC334534D633DE33E633F033FA330434EB
:1002E00013341D344534273431343B344E414E49A8
:1002F0004E495459494E46CDCCCC3D0AD7233C17E4
:10030000B7D13877CC2B329595E6241FB14F0A0030
:100310000020410000C84200401C4620BCBE4CCA20
:100320001B0E5AAEC59D7400407A10F35A00A0729D
:100330004E18090010A5D4E80000E8764817000020
:10034000E40B54020000CA9A3B000000E1F50500EE
:100350000080969800000040420F000000A0860137
:10036000000000102700000000E803000000006407
:1003700000000000000A0000000000010000000072
:10038000002C76D888DC674F0823DFC1DFAE59E147
:10039000B1B796E5E3E453C63AE651997696E8E6B6
:1003A000C28426EB898C9B62ED407C6FFCEFBC9C89
:1003B0009F40F2BAA56FA5F490055A2AF75C936B9B
:1003C0006CF9676DC11BFCE0E40D47FEF520E6B556
:1003D00000D0ED902E0300943577050080841E0830
:1003E0000000204E0A000000C80C333333330F984E
:1003F0006E12831141EF8D2114893BE65516CFFE15
:10040000E6DB18D1844B381BF77C1D901DA4BBE4A0
:1004100024203284725E228100C9F124ECA1E53DE2
:100420002700000A0B02090C0D0E08070304010047
:1004300000000000000000000000000000000000BC
:100440000000000000000000000000000012111079
:10045000000000000000000000000000000000009C
:100460000000000000000000002100240027002AF6
:10047000002D003000330001010000040107010AD3
:100480000100002200250028002B002E003100343E
:100490000002010000050108010B010000200023FB
:1004A00000260029002C002F00320000010000036C
:1004B00001060109010505050507050808080802E8
:1004C0000202020A0A0808040404040101010101ED
:1004D0000101010303030303030303040707070CDC
:1004E0000C0C0C0C0C0C0C02020202060606060692
:1004F0000606060B0B0B0B0B0B0B0B01021020203F
:100500000808102040102040800201020108040267
:1005100001010204081020408080402010080402DD
:100520000180040201804020100804020108040236
:10053000010102040810204080010204081020403C
:1005400080007A47754711241FBECFEFD1E2DEBF8E
:10055000CDBF00E00CBF17E0A0E0B2E0E6E0F3EAB8
:1005600000E00BBF02C007900D92A234B107D9F78B
:100570002CE0A2E4B7E001C01D92A23FB207E1F770
:1005800012E0C2EAD2E000E006C021970109802F04
:10059000FE010E946550C13AD10780E00807A9F723
:1005A0000E942A3D0C9472512BCD2F923F924F9274
:1005B0005F926F927F928F929F92AF92BF92CF92F3
:1005C000DF92EF92FF920F931F93CF93DF93CDB7FC
:1005D000DEB7E6970FB6F894DEBF0FBECDBF1C01A5
:1005E0002A013B010B871C872D873E872E960EAD77
:1005F0001FAD2E97FC01EF59FD4F60817181828103
:1006000093810E94BB4D9B01AC01C301B2010E94CA
:100610001A4E0E9411506B8B7C8B8D8B9E8BF1013F
:10062000EB59FD4F60817181828193810E94BB4DA6
:100630009B01AC016B857C858D859E850E941A4E41
:100640000E9411506B8F7C8F8D8F9E8FF101E75927
:10065000FD4F60817181828193810E94BB4D9B011E
:10066000AC01C701B6010E941A4E0E9411506F8F53
:1006700078A389A39AA30E941E106B877C878D871D
:100680009E87F101EE51FE4F118210823296118247
:1006900010823E96A114B10461F0C501A0E0B0E063
:1006A000408151816281738184179507A607B7073E
:1006B00014F0A080B180F101EA50FE4F8114910442
:1006C00061F0C401A0E0B0E040815181628173819A
:1006D00084179507A607B70714F080809180F10171
:1006E000E650FE4F0115110561F0C801A0E0B0E031
:1006F000408151816281738184179507A607B707EE
:1007000014F000811181310120E1620E711CC501DC
:10071000A0E0B0E0F10180A791A7A2A7B3A72101B3
:10072000FAE84F0E511CA12CB12CD20158968D9293
:100730009D92AD92BC925B974101BCEF8B1ABEEFCC
:100740009B0A20E030E0F401008F118F228F338F5D
:100750000E94D3180E94D3180E94D3180E94D31865
:1007600040914A0750914B0760914C0770914D079B
:100770004BAB5CAB6DAB7EAB0E94D31880914E0748
:1007800090914F07A0915007B09151078F87988B98
:10079000A98BBA8B0E94D318A0905207B090530730
:1007A000C0905407D0905507F101E359FD4F1082D6
:1007B0001182128213823496108211821282138265
:1007C0003496108211821282138234961182108222
:1007D00032961182108232961182108232964BA983
:1007E0005CA96DA97EA9408351836283738334968B
:1007F0008F859889A989BA8980839183A283B383DD
:100800003496A082B182C282D3822F96EFAC2F970A
:100810000B891C892D893E89C3010E949626882355
:10082000F9F085E393E00E94E33B8FEE95E00E94B0
:10083000E33BF101EE5AFF4F608171818281938128
:10084000E15FFD4F20813181428153810E94E74E5B
:10085000CA01B9010E942F3C0E94D3180E94DD17E3
:100860006096EFAC60970B8D1C8D2D8D3E8D4F8566
:10087000588969897A89C2010E9496268823F9F0ED
:1008800081E393E00E94E33B8FEF95E00E94E33B1E
:10089000F101E453FF4F6081718182819381E756BA
:1008A000FE4F20813181428153810E94E74ECA016F
:1008B000B9010E942F3C0E94D3180E94DD17619657
:1008C000EFAC61970F8D18A129A13AA1B601A5013E
:1008D000C4010E9496268823F9F08DE293E00E94DD
:1008E000E33B8FE096E00E94E33BF101EA5BFE4FC1
:1008F0006081718182819381ED5DFE4F2081318124
:10090000428153810E94E74ECA01B9010E942F3CE7
:100910000E94D3180E94DD17D10151961C92F1015B
:10092000E557FF4F1082E658FF4F1082C1010E9429
:100930008713C1010E948913C3010E94E42AC201E6
:100940000E94E42AC4010E94E42AF101E751FE4F0B
:10095000FCA3EBA381E090E0918380837101F5E13A
:10096000EF1AFEEFFF0AD7018D939C93810103518B
:100970001E4FF8019183808341E050E0B301C10133
:100980000E942B19D7014D915C91B201C1010E94C7
:100990002B19F80140815181B401C1010E942B192A
:1009A00011E0F101E253FD4F1083C3010E94812643
:1009B000C2010E948126C4010E94812664E670E083
:1009C00080E090E00E94E60FC1018A519E4FDC0159
:1009D0001C9311961C93A10148515E4FFA0110839C
:1009E0002F96FFAD2F97F1110FC060962FAD609736
:1009F000211105C061963FAD6197332339F1910113
:100A000021593F4FF90110826096FFAD6097F111B7
:100A100005C0910127513F4FF90110826196FFAD4A
:100A20006197F11105C091012D593E4FF9011082D6
:100A30002F962FAD2F97FC01208360963FAD6097D6
:100A40003C936196EFAD6197DA01EC93C3010E948C
:100A50003F28C2010E943F28C4010E943F28C301D1
:100A60000E949527C2010E949527C4010E949527E4
:100A70000E94D318DC011C968C918F87A12CB12C7D
:100A8000F101EA51FE4FFC8BEB8B910129513E4F56
:100A90003C8F2B8FA10148515E4F58A34F8FC1014E
:100AA00087519E4F9CA78BA7D101A551BE4FBEA7D2
:100AB000ADA73796F8ABEFA7255731403AA729A73E
:100AC0004F535F4F5AAB49AB815291409EA38DA3C8
:100AD000A95AB109B8A7AFA3EB89FC89808181111C
:100AE0000BC0AB8DBC8D8C91811106C0EF8DF8A130
:100AF0008081882309F44EC3FF85F1114BC34BA5B8
:100B00005CA5B301C1010E9482194DA55EA5B20189
:100B1000C1010E9482194FA558A9B401C1010E94C8
:100B20008219C3010E94FF27C2010E94FF27C4014E
:100B30000E94FF27E9A5FAA58081882321F1C3013E
:100B40000E943F28A9A9BAA98C918823C9F0610104
:100B5000B3E6CB1ABDEFDB0A7101E2E4EE1AEDEF6A
:100B6000FE0A810105571D4F910121583D4FA101FA
:100B700043595D4FB10162587E4FC3010E94CB12B1
:100B8000A9A5BAA51C92F101E451FF4F80818823E9
:100B900031F1C2010E943F28F101E655FD4F8081ED
:100BA0008823C9F06101BFE5CB1ABDEFDB0A7101F3
:100BB000E0E4EE1AEDEFFE0A810101571D4F9101AD
:100BC0002D573D4FA1014F585D4FB10164567E4FE7
:100BD000C2010E94CB12F101E451FF4F1082F101DA
:100BE000EA59FE4F8081882331F1C4010E943F28D9
:100BF000F101E555FD4F80818823C9F06101FBE5D6
:100C0000CF1AFDEFDF0A71012EE3E21A2DEFF20A8F
:100C100081010D561D4F910129573D4FA1014B58A0
:100C20005D4FB10166547E4FC4010E94CB12F101A9
:100C3000EA59FE4F1082810101591F4FD8018C9152
:100C4000882309F43CC0F101E956FD4F60817181B0
:100C5000072E000C880B990B0E94BB4D9B01AC0129
:100C6000F101E359FD4F60817181828193810E947E
:100C70004250181624F5D8011C9264E274E08101F8
:100C800008521E4FC8018ED76BED74E0C8018AD799
:100C90006CE973E0C80186D72F96BFAD2F97BB23B1
:100CA00009F47AC3F101E258FE4F108A118A128AC0
:100CB000138AE053F1401082118212821382810163
:100CC00007511F4FF8018081882309F43CC0E0558B
:100CD000FE4F60817181072E000C880B990B0E94DA
:100CE000BB4D9B01AC01F101EF58FD4F608171815B
:100CF000828193810E94425018162CF5F8011082CF
:100D000064E274E0810108521E4FC8014BD763E0D2
:100D100075E0C80147D76CE973E0C80143D7609616
:100D2000FFAD6097FF2309F43BC3F101E456FE4F8A
:100D3000108A118A128A138AADA1BEA11D921D923A
:100D40001D921C92139781010D591E4FF80180814D
:100D5000882309F43CC0E85CFE4F60817181072E56
:100D6000000C880B990B0E94BB4D9B01AC01F1015B
:100D7000EB58FD4F60817181828193810E944250C6
:100D800018162CF5D8011C9264E274E08101085217
:100D90001E4FC80107D76BE275E0C80103D76CE9A5
:100DA00073E0C801FFD66196BFAD6197BB2309F41C
:100DB000FBC2F101E654FE4F108A118A128A138A8F
:100DC000AFA1B8A51D921D921D921C92139760E0D1
:100DD000C3010E940E27882369F0F101E25BFF4FF7
:100DE0001082118212821382E05DFE4F108A118AF6
:100DF000128A138A60E0C2010E940E27882369F0DC
:100E0000EDA1FEA11082118212821382F101E4563B
:100E1000FE4F108A118A128A138A60E0C4010E9470
:100E20000E27882371F0AFA1B8A51D921D921D92C7
:100E30001C921397F101E654FE4F108A118A128A10
:100E4000138AF101E159FF4F8081EB89FC8980838E
:100E5000F101E751FF4F8081AB8DBC8D8C93E6583B
:100E6000FF4F8081EF8DF8A18083F101E25BFF4F9E
:100E700020813181428153812F83388749875A8766
:100E8000ADA1BEA14D915D916D917C91EFA1F8A5B1
:100E9000C080D180E280F3804BAB5CAB6DAB7EABAE
:100EA0000E94D3188F819885A985BA8580934A07B7
:100EB00090934B07A0934C07B0934D070E94D31813
:100EC0004BA95CA96DA97EA940934E0750934F078B
:100ED00060935007709351070E94D318C092520735
:100EE000D0925307E0925407F0925507C1010E9437
:100EF0008713AB89BC898C91882309F44AC00E946E
:100F00001E102B853C854D855E856217730784070F
:100F1000950760F40E941E102B853C854D855E85EB
:100F20006217730784079507A0F51EC00E941E1064
:100F30006B017C012B853C854D855E85C21AD30AE9
:100F4000E40AF50AF101EB5AFD4F2081318142811B
:100F50005381A8EEB3E00E94034F6C157D058E050A
:100F60009F0508F425C2D6CF0E941E106B017C019C
:100F7000F101EB5AFD4F2081318142815381A8EE6E
:100F8000B3E00E94034F6C157D058E059F0508F4A4
:100F90000FC2AB8DBC8D8C91882309F44AC00E948E
:100FA0001E102B853C854D855E856217730784076F
:100FB000950760F40E941E102B853C854D855E854B
:100FC0006217730784079507A0F51EC00E941E10C4
:100FD0006B017C012B853C854D855E85C21AD30A49
:100FE000E40AF50AF101E75AFD4F2081318142817F
:100FF0005381A8EEB3E00E94034F6C157D058E056A
:101000009F0508F4E8C1D6CF0E941E106B017C0139
:10101000F101E75AFD4F2081318142815381A8EED1
:10102000B3E00E94034F6C157D058E059F0508F403
:10103000D2C1AF8DB8A18C91882309F446C0FED7E8
:101040002B853C854D855E85621773078407950760
:1010500058F4F4D72B853C854D855E856217730760
:101060008407950790F51DC0E9D76B017C012B859E
:101070003C854D855E85C21AD30AE40AF50AF10162
:10108000E35AFD4F2081318142815381A8EEB3E0C4
:101090000E94034F6C157D058E059F0508F4AEC1B7
:1010A000D8CFCCD76B017C01F101E35AFD4F2081F1
:1010B000318142815381A8EEB3E00E94034F6C1549
:1010C0007D058E059F0508F499C188EA9BE026D32B
:1010D0001816190674F588EA9BE0FED28F7D8534D8
:1010E000910539F56DE974E0C10188529E4F5AD5DA
:1010F00082E693E00E94E33B0E94D3180E94DD1732
:10110000F101E159FF4F1082E658FF4F1082E65877
:10111000FF4F1082AB89BC891C92EB8DFC8D108235
:10112000AF8DB8A11C92B1E0BF87AA24A394B12CC3
:1011300003C0A114B10479F062EB74E0C1018852DC
:101140009E4F30D5EB89FC891082AB8DBC8D1C92F3
:10115000EF8DF8A11082C1010E94993BF101EC5181
:10116000FE4F808191810196918380838D329140E1
:101170000CF4B2CCD101A452BE4F8D919C91119729
:10118000892B09F0A9CC14968D919C91892B09F497
:1011900048C1A2CC810104521E4FD8018D919C916F
:1011A000892B21F0C1010E94993BF7CF82EC94E09A
:1011B0000E94E33B2F96BFAD2F97BB2309F1A114EB
:1011C000B104F1F4EF85E11140C08DE193E00E949C
:1011D000E33B0E94D3180E94DD176096FFAD609735
:1011E000FF2371F189E193E00E94E33B0E94D31851
:1011F0000E94DD1761962FAD6197211118C025C09F
:1012000060963FAD6097332339F0A114B10421F407
:101210004F8541111AC0E6CF61965FAD61975523A6
:10122000A1F0A114B10489F48F8581110EC085E16C
:1012300093E00E94E33B0E94D3180E94DD1705C093
:101240006196EFAD6197E111F2CF85E090E0ABA13F
:10125000BCA18D939C93910125513E4F3C872B87D8
:10126000D9018D939C93810103511E4FF801918305
:10127000808345E050E0B301C1010E942B19AB858A
:10128000BC854D915C91B201C1010E942B19F801FE
:1012900040815181B401C1010E942B19C1010E94FA
:1012A0008B13F101E25BFF4F4081518162817381B9
:1012B000E658FF4F80819181A281B3818F8B988FF7
:1012C000A98FBA8FE658FF4FC080D180E280F380AB
:1012D0004BAB5CAB6DAB7EAB0E94D3184BA95CA94A
:1012E0006DA97EA940934A0750934B0760934C0722
:1012F00070934D070E94D3182F89388D498D5A8DD0
:1013000020934E0730934F07409350075093510757
:101310000E94D318C0925207D0925307E09254070C
:10132000F0925507C1010E948713C1010E948913E1
:101330000E94D3180E943018C1010E94BA19ABA1B3
:10134000BCA11D921C92EB85FC8511821082D801F4
:101350001D921C9240E050E0B301C1010E942B1984
:10136000EB85FC8540815181B201C1010E942B199E
:10137000D8014D915C91B401C1010E942B19C101AA
:101380000E948B13BF85BB2309F43DC10E94D31873
:1013900021E0FC01248737C1AA24A394B12C8FCC6F
:1013A000AA24A394B12CCFCCAA24A394B12C0FCD02
:1013B00069E273E0810108521E4FC801F3D36CE962
:1013C00073E0C801EFD363E575E0C801EBD322E019
:1013D000A22EB12CDECD65E273E0810108521E4FD2
:1013E000C801E0D36CE973E0C801DCD368E675E0BE
:1013F000C801D8D392E0A92EB12C1BCE61E273E0D4
:10140000810108521E4FC801CDD36CE973E0C801B9
:10141000C9D36DE775E0C801C5D382E0A82EB12C11
:1014200054CE11821082F101EE51FE4F80819181E4
:10143000009741F46EE573E0810108521E4FC80128
:10144000B1D3BDC0019709F0CAC00E94D3188C0166
:10145000FC0180819181A281B381181619061A06B8
:101460001B0644F081E090E0A0E0B0E0808391832F
:10147000A283B383F80184819581A681B781181670
:1014800019061A061B0644F081E090E0A0E0B0E0E7
:1014900084839583A683B783F80180859185A2858F
:1014A000B385181619061A061B0644F081E090E071
:1014B000A0E0B0E080879187A287B3876EE973E0F0
:1014C000CE010196ADD36EEB74E0CE0101966AD3E6
:1014D0006FEE75E0CE01019665D360914A07709179
:1014E0004B0780914C0790914D070E94BB4D6B01BB
:1014F0007C01D8016D917D918D919C910E94BB4D95
:101500009B01AC01C701B6010E94A94FAB01BC0110
:10151000CE01019617D36FEF75E0CE01019642D34D
:1015200060914E0770914F0780915007909151073D
:101530000E94BB4D6B017C01F8016481758186813D
:1015400097810E94BB4D9B01AC01C701B6010E946F
:10155000A94FAB01BC01CE010196F4D26FE076E059
:10156000CE0101961FD3609152077091530780916D
:101570005407909155070E94BB4D6B017C01D80127
:1015800018966D917D918D919C911B970E94BB4DFA
:101590009B01AC01C701B6010E94A94FAB01BC0180
:1015A000CE010196CFD2BE016F5F7F4F81010852FD
:1015B0001E4FC80105D389819A810E94A3480E94C9
:1015C000D318BC01CE0101960E949717BE016F5F30
:1015D0007F4FC801F5D289819A810E94A348F10109
:1015E000EE51FE4F808191810196823091051CF46D
:1015F0009183808302C011821082F101E052FE4F7C
:101600001182108269CA80ED94E00E94E33BC5011B
:101610000E94563C8CE993E00E94E33B0E94D31861
:10162000B0924507A0924407C501E6960FB6F8941C
:10163000DEBF0FBECDBFDF91CF911F910F91FF9005
:10164000EF90DF90CF90BF90AF909F908F907F9062
:101650006F905F904F903F902F900895CF92DF92C0
:10166000EF92FF920F931F93CF93DF936C017A0158
:101670008B01C0E0D0E0CE15DF0589F0D8016D9177
:101680008D01D601ED91FC910190F081E02DC60114
:101690001995892B11F47E0102C02196ECCFC70168
:1016A000DF91CF911F910F91FF90EF90DF90CF903E
:1016B0000895089580E090E00895FC01538D448DD5
:1016C000252F30E0842F90E0821B930B541710F0ED
:1016D000CF96089501970895FC01918D828D9817FA
:1016E00061F0828DDF01A80FB11D5D968C91928D06
:1016F0009F5F9F73928F90E008958FEF9FEF089503
:10170000FC01918D828D981731F0828DE80FF11DCB
:10171000858D90E008958FEF9FEF0895FC01918DE6
:10172000228D892F90E0805C9F4F821B91098F73DF
:101730009927089588EA9BE0F1DF21E0892B09F4DD
:1017400020E0822F0895FC01848DDF01A80FB11DD8
:10175000A35ABF4F2C91848D90E001968F739927E7
:10176000848FA689B7892C93A089B1898C918064D4
:101770008C93938D848D981306C00288F389E02D95
:1017800080818F7D80830895EF92FF920F931F9346
:10179000CF93DF93EC0181E0888F9B8D8C8D981324
:1017A00005C0E889F989808185FD23C0F62E0B8D5F
:1017B00010E00F5F1F4F0F731127E02E8C8DE81282
:1017C0000BC00FB607FCFACFE889F989808185FF45
:1017D000F5CFCE01B8DFF2CF8B8DFE01E80FF11D02
:1017E000E35AFF4FF0820B8FEA89FB898081806288
:1017F00007C0EE89FF896083E889F9898081806468
:10180000808381E090E0DF91CF911F910F91FF9055
:10181000EF900895CF93DF93EC01888D8823C1F07A
:10182000EA89FB89808185FD05C0A889B9898C91E9
:1018300086FD0EC00FB607FCF5CF808185FFF2CF85
:10184000A889B9898C9185FFEDCFCE017CDFE8CFE7
:10185000DF91CF91089580E090E0892B19F06ADF45
:10186000811125C080E090E0892B41F080E090E07C
:10187000892B21F00E94000081111CC080E090E0C3
:10188000892B41F080E090E0892B21F00E9400003C
:10189000811113C080E090E0892BA1F080E090E0FE
:1018A000892B81F00E94000081110AC008950E94D6
:1018B0000000D8CF0E940000E1CF0E940000EACFD4
:1018C0000C940000089590E0FC013197E231F1059D
:1018D00008F04EC08827EE58FF4F8F4F0C9465508C
:1018E000809180008F7703C0809180008F7D8093EE
:1018F0008000089580918000877FF9CF84B58F772D
:1019000002C084B58F7D84BD08958091B0008F772B
:1019100003C08091B0008F7D8093B00008958091C6
:1019200090008F7707C0809190008F7D03C08091D9
:101930009000877F8093900008958091A0008F771A
:1019400007C08091A0008F7D03C08091A000877F99
:101950008093A0000895809120018F7707C0809127
:1019600020018F7D03C080912001877F809320011B
:1019700008953FB7F89480918F0B9091900BA091B0
:10198000910BB091920B26B5A89B05C02F3F19F083
:101990000196A11DB11D3FBFBA2FA92F982F8827EF
:1019A000820F911DA11DB11DBC01CD0142E0660F4A
:1019B000771F881F991F4A95D1F708950E945551A6
:1019C0000C94A3480C94A3480F931F93CF93DF93D9
:1019D000EC0188819981009729F02A813B812617A3
:1019E000370788F48B016F5F7F4F0E946D5000971F
:1019F00061F0998388831B830A832C813D81232B8B
:101A000011F4FC01108281E001C080E0DF91CF91F0
:101A10001F910F9108958F929F92AF92BF92CF9294
:101A2000DF92EF92FF920F931F930E94271762E0BD
:101A300070E00E94C536892BD1F40E94271721E05F
:101A40002F931F921F921F921F92812C912CA12CD9
:101A5000B12CC12CD12C760197018601B701A601CA
:101A60000E94D5020F900F900F900F900F9080E082
:101A700090E01F910F91FF90EF90DF90CF90BF907B
:101A8000AF909F908F9008958F929F92AF92BF9248
:101A9000CF92DF92EF92FF920F931F930E9427172E
:101AA0001F9221E02F931F921F921F92812C912C45
:101AB000A12CB12CC12CD12C760197018601B70144
:101AC000A6010E94D5020F900F900F900F900F90DB
:101AD00080E090E01F910F91FF90EF90DF90CF900A
:101AE000BF90AF909F908F900895EF92FF920F93C9
:101AF0001F93CF93DF93FC0124813581611571051C
:101B000011F480E018C041155105A1F07B01EC01F2
:101B10008A01020F131FB80157DF882391F3288130
:101B200039818C819D81B701820F931F0E946B5177
:101B30001D830C8381E0DF91CF911F910F91FF9066
:101B4000EF900895EF92FF920F931F93CF93DF933F
:101B5000CDB7DEB764970FB6F894DEBF0FBECDBF2A
:101B60007C01CB01BA018E010F5F1F4F22E044E0E0
:101B70000E94EF47BC01FC0101900020E9F731977A
:101B8000AF01481B590BC701B0DF64960FB6F8943C
:101B9000DEBF0FBECDBFDF91CF911F910F91FF90A0
:101BA000EF9008956115710549F0FB010190002047
:101BB000E9F73197AF01461B570B97CF80E00895A7
:101BC000FB0144815581608171818FCFEF92FF923B
:101BD0000F931F93CF93DF93EC017B018A01BA012E
:101BE000F3DE2881398181110DC02115310519F0ED
:101BF000C9010E94A348198218821D821C821B827F
:101C00001A8206C01D830C83B701C9010E946B5163
:101C1000CE01DF91CF911F910F91FF90EF9008952A
:101C2000FC011182108213821282158214826115C6
:101C3000710549F0FB0101900020E9F73197AF01F0
:101C4000461B570BC3CF08951F920F920FB60F92EA
:101C500011240BB60F922F933F934F935F936F9383
:101C60007F938F939F93AF93BF93EF93FF9388EAF4
:101C70009BE069DDFF91EF91BF91AF919F918F91B3
:101C80007F916F915F914F913F912F910F900BBE7C
:101C90000F900FBE0F901F9018951F920F920FB6C6
:101CA0000F9211240BB60F922F938F939F93EF9364
:101CB000FF93E091B80BF091B90B8081E091BE0BDE
:101CC000F091BF0B82FD12C090818091C10B8F5F9C
:101CD0008F732091C20B821751F0E091C10BF0E09D
:101CE000E855F44F958F8093C10B01C08081FF911F
:101CF000EF919F918F912F910F900BBE0F900FBE80
:101D00000F901F901895CF93DF93282F30E0F901A3
:101D1000EF5DFB4F8491F901E550FB4FD491F90140
:101D2000EB54FB4FC491CC2389F08111CCDDEC2F17
:101D3000F0E0EE0FFF1FE556FB4FA591B491EC913B
:101D4000ED2381E090E021F480E002C080E090E0AB
:101D5000DF91CF9108951F93CF93DF93282F30E029
:101D6000F901EF5DFB4F8491F901E550FB4FD491F0
:101D7000F901EB54FB4FC491CC23C1F0162F811114
:101D8000A2DDEC2FF0E0EE0FFF1FEF57FB4FA59108
:101D9000B4918FB7F894111105C09C91ED2FE09587
:101DA000E92302C0EC91ED2BEC938FBFDF91CF9133
:101DB0001F910895CF92DF92EF92FF920F931F939E
:101DC000CF93DF936C018B017A01EC01CA57D44F9A
:101DD000888187FF04C0FB011182108224C08CE03F
:101DE0008C9D90018D9D300D11248881A901480F93
:101DF000511D87FD5A958091DD0C90E048175907D9
:101E000094F48881A901480F511D87FD5A95CA0194
:101E1000FA01EE0FFF1F8E0F9F1FFC01E35BF34FD4
:101E2000808186FD19C088818F5F88838CE08C9DBE
:101E300090018D9D300D11248881A901480F511DFD
:101E400087FD5A958091DD0C90E048175907B4F44E
:101E500088818C303CF112C08881280F311D87FDAC
:101E60003A95F901EE0FFF1F2E0F3F1FF901E35BBB
:101E7000F34F808160E08F736EDFD5CFF8018081F2
:101E80009181049680349C4918F480E49CE904C054
:101E9000F801808191810496F701918380838FEF0F
:101EA000888344C0F801408151818881B901680F5D
:101EB000711D87FD7A95CB01FB01EE0FFF1F8E0F81
:101EC0009F1FFC01E35BF34F81819281840F951F7B
:101ED000F701918380838881A901480F511D87FDF7
:101EE0005A95CA01FA01EE0FFF1F8E0F9F1FFC01CA
:101EF000E35BF34F808186FF19C08881280F311D75
:101F000087FD3A95F901EE0FFF1F2E0F3F1FF901D4
:101F1000E35BF34F808161E08F73DF91CF911F917D
:101F20000F91FF90EF90DF90CF9015CFDF91CF9181
:101F30001F910F91FF90EF90DF90CF900895CF9376
:101F4000DF9390E0FC01E550FB4F2491FC01EB5442
:101F5000FB4F8491882361F190E0880F991FFC0169
:101F6000E959FB4FC591D491FC01EF57FB4FA59167
:101F7000B491611109C09FB7F8948881209582239C
:101F80008883EC912E230BC0623061F49FB7F894E4
:101F90003881822F809583238883EC912E2B2C937C
:101FA0009FBF06C08FB7F894E8812E2B28838FBF80
:101FB000DF91CF9108958230910538F0880F991FF5
:101FC000880F991F05970197F1F708958F929F92B7
:101FD000AF92BF92CF92DF92EF92FF926B017C01A2
:101FE000C8DC4B015C01C114D104E104F104E9F047
:101FF000C0DCDC01CB0188199909AA09BB09883E1C
:102000009340A105B10578F321E0C21AD108E10897
:10201000F10888EE880E83E0981EA11CB11CC11443
:10202000D104E104F10421F7DECFFF90EF90DF90BF
:10203000CF90BF90AF909F908F9008952FB7F89456
:1020400060918B0B70918C0B80918D0B90918E0B0E
:102050002FBF08951F920F920FB60F9211242F9346
:102060003F938F939F93AF93BF9380918B0B9091EE
:102070008C0BA0918D0BB0918E0B30918A0B23E0CD
:10208000230F2D3720F40196A11DB11D05C026E8B0
:10209000230F0296A11DB11D20938A0B80938B0BF9
:1020A00090938C0BA0938D0BB0938E0B80918F0B24
:1020B0009091900BA091910BB091920B0196A11D64
:1020C000B11D80938F0B9093900BA093910BB093C5
:1020D000920BBF91AF919F918F913F912F910F9054
:1020E0000FBE0F901F901895CF92DF92EF92FF9244
:1020F000CF93DF93EC01603282E078070CF03DC0B3
:1021000077FD06C0653B71052CF064EB70E002C002
:1021100060E070E0898128E830E06901C81AD108E0
:1021200087FDD394CC0CDD1CCC0CDD1C0D2C000CDD
:10213000EE08FF088A8128E532E0281B310987FD77
:102140003395220F331F220F331FC901330FAA0B00
:10215000BB0B9C01AD012C193D094E095F09DB0148
:102160000E940D4F24EB30E040E050E00E94E74E2B
:10217000C20ED31EE41EF51EB6018881803380F5A1
:10218000998148E850E0491B510997FD5395440F48
:10219000551F440F551F6417750784F09A8128E571
:1021A00032E0291B310997FD3395220F331F220F8F
:1021B000331FAB01261737070CF4A9014250510910
:1021C000440F551F2FB7F89490E0FC01EE0FFF1F4E
:1021D0008E0F9F1FFC01E35BF34F528341832FBFA0
:1021E000DF91CF91FF90EF90DF90CF9008951F93F4
:1021F000CF93DF93EC01162F8881803308F04DC018
:1022000061E0812F9CDE8881E82FF0E09F01220FA2
:10221000331FE20FF31FE35BF34F1F739081907C3A
:10222000192B108319821A826CE00E9459509CE08D
:10223000899FB001112440E050E09A01260F371F1A
:10224000F901EE0FFF1F2E0F3F1FF901E35BF34F64
:10225000908196FD16C04F5F5F4F4C30510569F776
:10226000813001F51092800082E08093810010920D
:10227000850010928400B19A80916F0082608093F3
:102280006F00E881F0E0CF01880F991FE80FF91F78
:10229000E35BF34F8081806480838881DF91CF91FD
:1022A0001F910895823061F4109290008093910004
:1022B000109295001092940088BB80937100E1CF3A
:1022C000833069F41092A00082E08093A100109204
:1022D000A5001092A40089BB80937200D2CF811117
:1022E000D0CF1092200182E080932101109225012D
:1022F000109224018ABB80937300C3CF1F920F9268
:102300000FB60F9211240BB60F922F933F934F935A
:102310005F936F937F938F939F93AF93BF93EF934D
:10232000FF9348E251E064E271E080E090E042DD3A
:10233000FF91EF91BF91AF919F918F917F916F919D
:102340005F914F913F912F910F900BBE0F900FBE59
:102350000F901F9018951F920F920FB60F92112495
:102360000BB60F922F933F934F935F936F937F938F
:102370008F939F93AF93BF93EF93FF9348EA50E0FF
:1023800064EA70E083E090E015DDFF91EF91BF918A
:10239000AF919F918F917F916F915F914F913F91FD
:1023A0002F910F900BBE0F900FBE0F901F9018959E
:1023B0001F920F920FB60F9211240BB60F922F930C
:1023C0003F934F935F936F937F938F939F93AF93BD
:1023D000BF93EF93FF9348E950E064E970E082E037
:1023E00090E0E8DCFF91EF91BF91AF919F918F91C9
:1023F0007F916F915F914F913F912F910F900BBE05
:102400000F900FBE0F901F9018951F920F920FB64E
:102410000F9211240BB60F922F933F934F935F931C
:102420006F937F938F939F93AF93BF93EF93FF939C
:1024300048E850E064E870E081E090E0BBDCFF91A8
:10244000EF91BF91AF919F918F917F916F915F912C
:102450004F913F912F910F900BBE0F900FBE0F9099
:102460001F90189508950F931F93CF93DF93FC014E
:102470002081318121153105D1F1EC01822F43DC1E
:1024800021E0892B09F420E02B876A85261729F0A3
:102490001E821F82188619860BC08E819F81A88597
:1024A000B9850196A11DB11D8E839F83A887B98729
:1024B0000E811F81288539858A819B81AC81BD81F0
:1024C000081719072A073B0794F081E068278881DD
:1024D00042DC0990D881C02D0E946D3540E050E06B
:1024E000BE01DF91CF911F910F910C94D732DF91F4
:1024F000CF911F910F910895CF92DF92EF92FF92AB
:102500000F931F93CF93DF937C016B018A01E90145
:102510000E944532F601EE0FFF1FEE0FFF1FEA5A31
:10252000F84F80819181F701918380830E94453229
:10253000000F111F000F111FF801EA5AF84F81E038
:10254000408151816281738141305105610571057E
:1025500009F080E0F70182870E944532CC0FDD1F31
:10256000CC0FDD1FCA5AD84F88819981AA81BB81BF
:10257000F70182839383A483B58316821782108622
:102580001186DF91CF911F910F91FF90EF90DF9017
:10259000CF90089508952F923F924F925F926F923D
:1025A0007F928F929F92AF92BF92CF92DF92EF92E3
:1025B000FF920F931F93CF93DF9300D000D0CDB73E
:1025C000DEB79E838D834B015A013A83298318011C
:1025D000FC82EB82FA01408051806280738020E0AF
:1025E00030E0A901C301B2010E944250181674F4F0
:1025F000F6012081318142815381C301B2010E94E1
:10260000444FF5016083718382839383ED81FE8162
:10261000E05AFF4F8081F401028D138DC088D1886C
:10262000E288F388F1014080518062807380D80194
:10263000A7019601882341F00E940D4F641575058E
:102640008605970544F023C00E940D4F4616570695
:1026500068067906E4F4F501408051806280738059
:1026600020E030E04AEF56E4C301B2010E94B54DCC
:1026700087FF0DC020E030E040E85FE3C301B20116
:102680000E94454FF5016083718382839383D80153
:10269000A70196010E940D4FF1016083718382832F
:1026A00093830D811E81025C1F4FF801808191810F
:1026B000A281B381E981FA8180839183A283B3836C
:1026C000EB81FC8180819181892B41F0C4010E94C2
:1026D0007736F801608371838283938326960FB6E1
:1026E000F894DEBF0FBECDBFDF91CF911F910F9148
:1026F000FF90EF90DF90CF90BF90AF909F908F9022
:102700007F906F905F904F903F902F9008954BD5A2
:1027100091C749D564C4CF93DF93EC01FC01E25328
:10272000FD4F1082EE58F1098081811104C0CE0165
:1027300040960E946D26FE01EF5BFD4F8081811166
:1027400005C0CE0186579F4F0E946D26FE01EE5BAD
:10275000FD4F8081811105C0CE018C5F9E4F0E948C
:102760006D2664E670E080E090E0DF91CF912ECCA2
:10277000662319F08DEA93E002C086EA93E00C9498
:10278000E33B0C94A3480C94A3488F929F92AF9282
:10279000BF92CF92DF92EF92FF920F931F93CF934E
:1027A000DF93EC018AE190E09E8B8D8B8BE190E0D2
:1027B000988F8F8B89E190E09A8F898F8FE090E0DE
:1027C0009C8F8B8F8EE190E09E8F8D8F8EE090E0BE
:1027D00098A38F8F85E490E09AA389A384E490E086
:1027E0009CA38BA3FE01E657FF4F80E290E0968307
:1027F000858381E290E0908787838FE190E09287E4
:1028000081871486138616861586108A178683E4B8
:1028100090E0928B818B82E490E0948B838BE658DE
:10282000FF4F83E290E09683858384E290E0908777
:10283000878382E290E092878187148613861686CA
:102840001586108A178681E490E0928B818B80E454
:1028500090E0948B838BEB51FF4F11821082329664
:1028600011821082329611821082CE010E94831D45
:10287000CE015CD76E0182E8C81A8EEFD80A882490
:102880008394912CF601958E848E7E01F4E6EF1AE6
:10289000FEEFFF0A84E090E0F701958F848F8E01B0
:1028A00006541E4F88E090E0F801958F848F80E1F8
:1028B00090E0F6019183808381E190E095838483A9
:1028C000AA24AA94BA2CB382A282B782A682C60195
:1028D0000E941136F601828580878385818787E192
:1028E00090E0F7019183808388E190E09583848371
:1028F000B382A282B782A682C7010E941136F70175
:1029000082858087838581878DE190E0F8019183BE
:1029100080838CE190E095838483B382A282B78226
:10292000A682C8010E941136F801828580878385BE
:102930008187E65FFE4F808191817297408151814E
:1029400062817381369720813181F601318F208F2A
:10295000448B558B668B778B019719F4B38EA28EBF
:1029600003C0F601938E828EFE01EA53FD4F8081F3
:102970009181709740815181628173813897208164
:102980003181F701318F208F448B558B668B778B8C
:10299000019719F48FEF9FEF03C081E090E0F701FA
:1029A000938F828FFE01E853FD4F808191813E9786
:1029B0004081518162817381C055DD4F2881398109
:1029C000F801318F208F448B558B668B778B019765
:1029D00019F48FEF9FEF03C081E090E0F801938F2F
:1029E000828FDF91CF911F910F91FF90EF90DF9039
:1029F000CF90BF90AF909F908F9008952F923F926D
:102A00004F925F926F927F928F929F92AF92BF92FE
:102A1000CF92DF92EF92FF920F931F93CF93DF93AA
:102A2000CDB7DEB7CA57D1090FB6F894DEBF0FBED7
:102A3000CDBF8C01FC01108211821282138214829C
:102A400015821682178210861186128613861486C6
:102A50001586168617862C01F0E14F0E511CC20117
:102A60000E94062B68018AE8C80ED11CC6010E948C
:102A7000062B7801ECEFEE1AEEEFFE0AC7010E947A
:102A8000062B3801F2E86F1AFEEF7F0AC3010E949D
:102A9000A136480184E6881A8EEF980AC4010E9484
:102AA000A1365801E6E4AE1AEEEFBE0AC5010E9457
:102AB000A1366EE973E0C80188529E4FB1D8F80183
:102AC000E252FE4F118210823296118210823296AB
:102AD00011821082329611821082329610823196C3
:102AE00010823196108231961182108232961182B4
:102AF00010823296118210823296108231961082A4
:102B0000319610823196108211821282138234968D
:102B100010821182128213823496108211821282E4
:102B2000138234961082118212821382349610829C
:102B300011821282138234961082118212821382C1
:102B4000349610821182128213823496108211827E
:102B5000128213823496108211821282138234966A
:102B60001082118212821382349610821182128294
:102B7000138234961082118212821382349610824C
:102B80001182128213823496108211821282138271
:102B900034961082118212821382349610823196FA
:102BA0001082319610823196108211821282138225
:102BB000349610821182128213823496108211820E
:102BC00012821382349610823196108231961082CE
:102BD0003196108231961082319610823196108291
:102BE0003196108231961082319610823196108281
:102BF0003196108231961082319610823196108271
:102C00003196108231961082319610823196108260
:102C10003196108231961082319610823196108250
:102C2000319610823196108211821282138234966C
:102C300010821182128213823496108211821282C3
:102C40001382D801AF59BD4F8CE0E9E3F3E0019066
:102C50000D928A95E1F7F801E359FD4F1082118238
:102C60001282138234961082118212821382349659
:102C7000108211821282138234961182108232964F
:102C80001182108232961182108232961082118245
:102C90001282138234961082118212821382349629
:102CA0001082118212821382349610821182128253
:102CB000138234961082118212821382349610820B
:102CC00011821282138234961182108232961182FE
:102CD00010823296118210823296108211821282F4
:102CE00013823496108211821282138234961082DB
:102CF000118212821382349610823196108231969C
:102D00001082319611821082329611821082329690
:102D100011821082329610821182128213823496AE
:102D200010821182128213823496108211821282D2
:102D3000138234961182108232961182108232965A
:102D40001182108232961182108232961182108284
:102D5000329611821082329611821082329611823E
:102D600010821801F2E32F1AFDEF3F0AF1011082E1
:102D7000CE0101960E94062B8AE7FE013196D20110
:102D800001900D928A95E1F7CE0101960E94062BE3
:102D90008AE7FE013196D60101900D928A95E1F7FE
:102DA000CE0101960E94062B8AE7FE013196D701DB
:102DB00001900D928A95E1F788E5F801808B89E50D
:102DC000F60180838AE5F7018083CE0101960E9497
:102DD000A1368EE1FE013196D30101900D928A95C4
:102DE000E1F7CE0101960E94A1368EE1FE013196F7
:102DF000D40101900D928A95E1F7CE0101960E94CF
:102E0000A1368EE1FE013196D50101900D928A9591
:102E1000E1F7C801BADCF1011082C658DF4F0FB6E6
:102E2000F894DEBF0FBECDBFDF91CF911F910F9100
:102E3000FF90EF90DF90CF90BF90AF909F908F90DA
:102E40007F906F905F904F903F902F900895CF9319
:102E5000DF9380919D0B90919E0B892B51F48FEC09
:102E600092E00E940E48EC01C9DDD0939E0BC09306
:102E70009D0B80919D0B90919E0BDF91CF910895BA
:102E80004F925F926F927F928F929F92AF92BF927A
:102E9000CF92DF92EF92FF920F931F93CF93DF9326
:102EA00000D01F92CDB7DEB7FB0116890789828853
:102EB0009388A684B784C284D384E484F58446804E
:102EC0005780608471844281538164817581498314
:102ED0005A836B837C83BBDF1F921F921F920F93D9
:102EE0001F939301820149815A816B817C810E94E9
:102EF000D5020F900F900F900F900F9080E090E010
:102F00000F900F900F900F90DF91CF911F910F9125
:102F1000FF90EF90DF90CF90BF90AF909F908F90F9
:102F20007F906F905F904F90089508950895EF926D
:102F3000FF920F931F93CF93DF93CDB7DEB72E97FA
:102F40000FB6F894DEBF0FBECDBF8C016EE973E003
:102F50000E94100E62E975E0C8010E94D20D6091D6
:102F600046077091470780914807909149072AE0EA
:102F7000AE014F5F5F4F7A010E947249F7010190E5
:102F80000020E9F73197AF014E195F09B701C80179
:102F90000E94750D6CE973E0C8010E94D20DC80152
:102FA0002E960FB6F894DEBF0FBECDBFDF91CF9146
:102FB0001F910F91FF90EF90089582E995E00E9494
:102FC000E33B6091460770914707809148079091D5
:102FD00049070E942F3C8CE993E00C94E33B0F934C
:102FE0001F93CF93DF93EC0185E995E00E94E33BCB
:102FF00089E995E00E94E33B07E91BE0F801608165
:10300000CE01B6DB8DE995E00E94E33BF8016181DA
:10301000CE01AEDB81EA95E00E94E33BF8016281DC
:10302000CE01A6DB85EA95E00E94E33BF8016381CF
:10303000CE019EDB89EA95E00E94E33BF8016481C2
:10304000CE0196DB8DEA95E00E94E33BF8016581B5
:10305000CE018EDBCE01DF91CF911F910F91ADCFCD
:10306000CF92DF92EF92FF92CF93DF93EC018881B2
:103070009981AA81BB81181619061A061B0644F00D
:1030800081E090E0A0E0B0E088839983AA83BB83CD
:103090008C819D81AE81BF81181619061A061B0608
:1030A00044F081E090E0A0E0B0E08C839D83AE83AB
:1030B000BF8388859985AA85BB85181619061A06C7
:1030C0001B0644F081E090E0A0E0B0E0888799879B
:1030D000AA87BB878EEB94E00E94E33B8FEE95E0DE
:1030E0000E94E33B60914A0770914B0780914C0727
:1030F00090914D070E94BB4D6B017C0168817981E5
:103100008A819B810E94BB4D9B01AC01C701B60126
:103110000E94A94F42E00E945B3C8FEF95E00E9425
:10312000E33B60914E0770914F078091500790915B
:1031300051070E94BB4D6B017C016C817D818E81AA
:103140009F810E94BB4D9B01AC01C701B6010E944B
:10315000A94F42E00E945B3C8FE096E00E94E33B77
:1031600060915207709153078091540790915507D1
:103170000E94BB4D6B017C01688579858A859B85A2
:103180000E94BB4D9B01AC01C701B6010E94A94F33
:1031900042E00E945B3CCE01DF91CF91FF90EF9027
:1031A000DF90CF900ACF8091950B9091960B892B51
:1031B00091F58DE090E00E940E48FC01148610927B
:1031C0004A0710924B0710924C0710924D0710922D
:1031D0004E0710924F07109250071092510710920D
:1031E00052071092530710925407109255071092ED
:1031F000940B1092930B109246071092470710926F
:10320000480710924907109245071092440790937F
:10321000960B8093950B8091950B9091960B08954A
:103220000F931F93CF93DF938B01EA0181E593E026
:103230000E94E33B8EE496E00E94E33BF80180812C
:103240000E94243CCE010E94563CADDFDF91CF911D
:103250001F910F91B2CECF92DF92EF92FF920F9318
:103260001F93CF93DF93CDB7DEB728970FB6F894AF
:10327000DEBF0FBECDBF8B016A0188529E4F7C011D
:103280006DE473E00E94D20D6EE476E0C7010E9407
:10329000D20DF801808189831A8241E050E08E01CD
:1032A0000F5F1F4FB801C7010E94750D4AE0B801BA
:1032B000C6010E946849F80101900020E9F73197A2
:1032C000AF01401B510BB801C7010E94750D6BDFA8
:1032D000BC01C8012CDEB801C7010E94E00D898144
:1032E0009A810E94A34828960FB6F894DEBF0FBEBD
:1032F000CDBFDF91CF911F910F91FF90EF90DF90A5
:10330000CF900895FC01DB01AD59BF4F8C9188230C
:1033100019F022E030E002C020E030E0DB01AB59E0
:10332000BF4F8C91882311F023E030E0DB01AC59D2
:10333000BF4F8C91882311F024E030E0DB01AA59C3
:10334000BF4F8C91882311F026E030E0DA018D9197
:103350009C918217930721F091E0121613060CF04E
:1033600090E0DA012D933C93992319F0A901CF0144
:1033700072CF08958F929F92AF92BF92CF92DF92B9
:10338000EF92FF920F931F93CF93DF93EC0189E4A9
:1033900093E00E94E33B8FEE95E00E94E33B6E01D9
:1033A00082E8C81A8EEFD80AC6010E9477360E94BA
:1033B000BB4D4B015C01FE01EF59FD4F60817181F6
:1033C000828193810E94BB4D9B01AC01C501B40178
:1033D0000E94A94F42E00E945B3C8FEF95E00E9463
:1033E000E33B7E01E4E6EE1AEEEFFE0AC7010E941F
:1033F00077360E94BB4D4B015C01FE01EB59FD4F3E
:1034000060817181828193810E94BB4D9B01AC01DF
:10341000C501B4010E94A94F42E00E945B3C8FE0CD
:1034200096E00E94E33B8E0106541E4FC8010E94A5
:1034300077360E94BB4D4B015C01C759DD4F688157
:1034400079818A819B810E94BB4D9B01AC01C501A2
:10345000B4010E94A94F42E00E945B3CA4DEADDDB6
:1034600085E493E00E94E33B8FEE95E00E94E33B0E
:10347000F601A28DB38D20893189428953890E943A
:103480000D4F0E942F3C8FEF95E00E94E33BF70128
:10349000A28DB38D20893189428953890E940D4FB5
:1034A0000E942F3C8FE096E00E94E33BF801A28D42
:1034B000B38D20893189428953890E940D4F0E9422
:1034C0002F3C71DEDF91CF911F910F91FF90EF9014
:1034D000DF90CF90BF90AF909F908F906ECD4F9226
:1034E0005F926F927F928F929F92AF92BF92CF9294
:1034F000DF92EF92FF920F931F93CF93DF9300D051
:103500001F92CDB7DEB70E944532409032085090EE
:10351000330860903408709035080E9445328090DE
:10352000360890903708A0903808B09039083BDEF4
:10353000C0904A07D0904B07E0904C07F0904D07A1
:1035400032DEC701B6010E94BB4D6B017C01C30195
:10355000B2010E94BB4D9B01AC01C701B6010E94A4
:10356000A94F2B013C0160914E0770914F0780914C
:103570005007909151070E94BB4D6B017C01C50122
:10358000B4010E94BB4D9B01AC01C701B6010E9472
:10359000A94FAB01BC0149835A836B837C8357DC01
:1035A0001F921F921F921F921F92812C912CA12C6F
:1035B000B12CC12CD12C760149815A816B817C813F
:1035C0008A019B01B301A2010E94D50240DC1F9237
:1035D0001F921F921F921F9297018601B301A201B1
:1035E0000E94D50234DC1F921F921F921F921F92DD
:1035F00097018601B701A6010E94D5020FB6F89483
:10360000DEBF0FBECDBF80E090E00F900F900F9017
:103610000F90DF91CF911F910F91FF90EF90DF906E
:10362000CF90BF90AF909F908F907F906F905F9062
:103630004F900895CF93DF9385E40E94830EEC01B1
:10364000B2DD91E0CD2B09F490E09093970B84E4E8
:103650000E94830EEC01A7DD91E0CD2B09F490E0F0
:103660009093980B83E40E94830EEC019CDD91E023
:10367000CD2B09F490E09093990B82E40E94830E85
:10368000EC0191DD91E0CD2B09F490E090939A0B41
:1036900081E40E94830EEC0186DD91E0CD2B09F4DC
:1036A00090E090939B0B80E40E94830EEC017BDD05
:1036B00091E0CD2B09F490E090939C0BDF91CF919A
:1036C0000895CF93DF93EC012AEC30E04BEC50E00F
:1036D00069EC70E00E947C122EEC30E04FEC50E080
:1036E0006DEC70E0CE010C960E947C1224ED30E06F
:1036F00045ED50E063ED70E0CE0148960E947C12EB
:1037000028ED30E049ED50E067ED70E0CE018496A1
:103710000E947C122EED30E04FED50E06DED70E038
:10372000CE01C096DF91CF910C947C122F923F92E4
:103730004F925F926F927F928F929F92AF92BF92C1
:10374000CF92DF92EF92FF920F931F93CF93DF936D
:10375000EC010E944532FE01E956FD4F80911209AD
:1037600090911309918380830E944532FE01E756B0
:10377000FD4F8091160990911709918380830E94D3
:103780004532FE01E556FD4F80911A0990911B09C3
:10379000918380830E9445328E0103561D4F6091B4
:1037A0003A0970913B0980913C0990913D090E9432
:1037B000BB4DF80160837183828393830E944532FD
:1037C0001E01FFE52F1AFDEF3F0A60913E0970913F
:1037D0003F0980914009909141090E94BB4DF10140
:1037E00060837183828393830E94453220E030E0BE
:1037F00048EC52E4F80160817181828193810E94DA
:10380000A94F2B013C0120E030E048EC52E4F101EB
:1038100060817181828193810E94A94F4B015C017B
:103820006091420970914309809144099091450942
:103830000E94BB4D20E030E048EC52E40E94A94FCA
:103840006B017C012AE037ED43E25CE3C301B20186
:103850000E94425018168CF420E030E046EC52E40E
:10386000C301B2010E94B54D87FD0FC0412C512C00
:1038700046EC642E42E4742E08C05AE0452E57ED03
:10388000552E53E2652E5CE3752EF801408251827D
:10389000628273822AE037ED43E25CE3C501B40142
:1038A0000E94425018168CF420E030E046EC52E4BE
:1038B000C501B4010E94B54D87FD0FC0812C912C2C
:1038C00026ECA22E22E4B22E08C03AE0832E37ED79
:1038D000932E33E2A32E3CE3B32EF101808291823A
:1038E000A282B3822AE037ED43E25CE3C701B6016E
:1038F0000E94425018168CF420E030E046EC52E46E
:10390000C701B6010E94B54D87FD0FC0C12CD12C57
:1039100086ECE82E82E4F82E08C09AE0C92E97EDD6
:10392000D92E93E2E92E9CE3F92EFE01EB55FD4FD3
:10393000C082D182E282F3820E9445328091FA08ED
:103940009091FB08FE01E455FD4F918380830E9416
:1039500045328091FE089091FF08FE01E255FD4F2F
:10396000918380830E9445328091020990910309DE
:10397000FE01E055FD4F918380830E944532809186
:10398000220990912309A0912409B0912509FE01F3
:10399000EE54FD4F80839183A283B3830E9445320E
:1039A0008091260990912709A0912809B0912909B1
:1039B000FE01EA54FD4F80839183A283B3830E946A
:1039C000453280912A0990912B09A0912C09B09140
:1039D0002D09FE01E654FD4F80839183A283B383BA
:1039E0000E94453280914A0990914B09FE01E254B0
:1039F000FD4F918380830E94453280914E099091C2
:103A00004F09FE01E054FD4F918380830E944532AF
:103A10008091520990915309FE01EE53FD4F91831D
:103A200080830E9445328091620990916309FE0172
:103A3000EC53FD4F918380830E944532809166094B
:103A400090916709FE01EA53FD4F918380830E94A4
:103A5000453280916A0990916B09FE01E853FD4F50
:103A6000918380830E9445328091EA089091EB080F
:103A7000A091EC08B091ED08FE01E755FD4F0197CC
:103A8000A105B10519F481E0808301C010820E9474
:103A900045328091EE089091EF08A091F008B09126
:103AA000F108FE01E655FD4F0197A105B10519F496
:103AB00081E0808301C010820E9445328091F2082B
:103AC0009091F308A091F408B091F508C555DD4F29
:103AD0000197A105B10519F481E0888301C018821E
:103AE000DF91CF911F910F91FF90EF90DF90CF90DA
:103AF000BF90AF909F908F907F906F905F904F900E
:103B00003F902F9008952F923F924F925F926F9225
:103B10007F928F929F92AF92BF92CF92DF92EF925D
:103B2000FF920F931F93CF93DF93CDB7DEB76097CC
:103B30000FB6F894DEBF0FBECDBF988B8F870E9463
:103B40004532EF85F889E151FE4F81E0409122082E
:103B5000509123086091240870912508452B462B2D
:103B6000472B09F480E080830E944532EF85F88975
:103B7000E051FE4F81E04091260850912708609166
:103B8000280870912908452B462B472B09F480E023
:103B900080830E944532EF85F889EF50FE4F81E027
:103BA00040912A0850912B0860912C0870912D08A3
:103BB000452B462B472B09F480E080830E94453239
:103BC0008091720890917308A0917408B091750863
:103BD000EF85F889EE50FE4F80839183A283B383F3
:103BE0000E9445328091760890917708A0917808DC
:103BF000B0917908EF85F889EA50FE4F8083918370
:103C0000A283B3830E94453280917A0890917B0809
:103C1000A0917C08B0917D08EF85F889E650FE4FB1
:103C200080839183A283B3830E94453280914A08A6
:103C300090914B08A0914C08B0914D08EF85F88900
:103C4000E65FFD4F80839183A283B3830E94453258
:103C500080914E0890914F08A0915008B091510862
:103C6000EF85F889E25FFD4F80839183A283B38360
:103C70000E9445328091520890915308A0915408B7
:103C8000B0915508EF85F889EE5EFD4F80839183F2
:103C9000A283B3830E94453280915A0890915B08B9
:103CA000A0915C08B0915D08EF85F889EA5EFD4F50
:103CB00080839183A283B3830E94453280915E0802
:103CC00090915F08A0916008B0916108EF85F88934
:103CD000E65EFD4F80839183A283B3830E944532C9
:103CE0008091620890916308A0916408B091650882
:103CF000EF85F889E25EFD4F80839183A283B383D1
:103D00000E9445328091FA079091FB07A091FC0731
:103D1000B091FD07EF85F889EE5DFD4F80839183BB
:103D2000A283B3830E9445328091FE079091FF07E2
:103D3000A0910008B0910108EF85F889EA5DFD4F78
:103D400080839183A283B3830E94453280910208CD
:103D500090910308A0910408B0910508EF85F889B7
:103D6000E65DFD4F80839183A283B3830E94453239
:103D7000EF85F889E25DFD4F81E02091D207309117
:103D8000D3072130310509F080E080830E9445325D
:103D9000EF85F889E15DFD4F81E02091D6073091F4
:103DA000D7072130310509F080E080830E94453239
:103DB000EF85F889E05DFD4F81E02091DA073091D1
:103DC000DB072130310509F080E080830E94453215
:103DD000EF85F889E45BFD4F81E04091AA0750919F
:103DE000AB076091AC077091AD07452B462B472B75
:103DF00009F480E080830E944532EF85F889E35B17
:103E0000FD4F81E04091AE075091AF076091B00740
:103E10007091B107452B462B472B09F480E0808336
:103E20000E944532EF85F889E25BFD4F81E04091C9
:103E3000B2075091B3076091B4077091B507452B55
:103E4000462B472B09F480E080830E944532EF85A2
:103E5000F889E15BFD4F81E0409182085091830831
:103E60006091840870918508452B462B472B09F4F7
:103E700080E080830E944532EF85F889E05BFD4F4A
:103E800081E0409186085091870860918808709180
:103E90008908452B462B472B09F480E080830E943C
:103EA0004532EF85F889EF5AFD4F81E040918A084D
:103EB00050918B0860918C0870918D08452B462B92
:103EC000472B09F480E080830E944532EF85F88912
:103ED000EE5AFD4F81E02091BA073091BB072130A7
:103EE000310509F080E080830E944532EF85F88932
:103EF000ED5AFD4F81E02091BE073091BF07213080
:103F0000310509F080E080830E944532EF85F88911
:103F1000EC5AFD4F81E02091C2073091C307213058
:103F2000310509F080E080830E944532809182074C
:103F300090918307A0918407B0918507EF85F88958
:103F4000EB5AFD4F80839183A283B3830E94453255
:103F50008091860790918707A0918807B091890783
:103F6000EF85F889E75AFD4F80839183A283B3835D
:103F70000E94453280918A0790918B07A0918C070F
:103F8000B0918D07EF85F889E35AFD4F80839183C7
:103F9000A283B3830E944532EF85F889E05CFD4F30
:103FA00081E040919207509193076091940770913E
:103FB0009507452B462B472B09F480E080830E9410
:103FC0004532EF85F889EF5BFD4F81E04091960720
:103FD000509197076091980770919907452B462B50
:103FE000472B09F480E080830E944532EF85F889F1
:103FF000EE5BFD4F81E040919A0750919B076091E5
:104000009C0770919D07452B462B472B09F480E0B8
:1040100080830E94453280918A0990918B09A091FA
:104020008C09B0918D09EF85F889EF5CFD4F808395
:104030009183A283B3830E94453280918E0990912F
:104040008F09A0919009B0919109EF85F889EB5CF7
:10405000FD4F80839183A283B3830E944532809178
:10406000920990919309A0919409B0919509EF85D7
:10407000F889E75CFD4F80839183A283B3830E941C
:104080004532EF85F889ED5BFD4F81E02091EA072D
:104090003091EB072130310509F080E08083EF8516
:1040A000F889EC5BFD4F1082EF85F889EB5BFD4FE3
:1040B00010820E944532EF85F889EA5BFD4F81E06E
:1040C0002091E6073091E7072130310509F080E0C3
:1040D0008083EF85F889E95BFD4F1082EF85F889D1
:1040E000E85BFD4F10820E944532EF85F889E75B5F
:1040F000FD4F81E020910A0830910B0821303105F5
:1041000009F080E080830E944532EF85F889E65B04
:10411000FD4F81E020910E0830910F0821303105CC
:1041200009F080E080830E944532EF85F889E55BE5
:10413000FD4F81E0209112083091130821303105A4
:1041400009F080E080830E944532EF85F889E35CC6
:10415000FD4F81E020919A0930919B092130310572
:1041600009F080E080830E944532EF85F889E25CA7
:10417000FD4F81E020919E0930919F09213031054A
:1041800009F080E080830E944532EF85F889E15C88
:10419000FD4F81E02091A2093091A3092130310522
:1041A00009F080E080830E9445320F8518890F59FD
:1041B0001D4F8091320890913308A0913408B0913E
:1041C0003508F80180839183A283B3830E9445322E
:1041D000EF84F888FBE9EF1AFDEFFF0A80913608BB
:1041E00090913708A0913808B0913908F701808381
:1041F0009183A283B3830E94453280913A089091C3
:104200003B08A0913C08B0913D082F85388927597B
:104210003D4FF90180839183A283B383F8014081EC
:10422000518162817381141615061606170644F033
:1042300041E050E060E070E040835183628373832B
:10424000F7014081518162817381141615061606AB
:10425000170644F041E050E060E070E04083518395
:1042600062837383181619061A061B064CF081E048
:1042700090E0A0E0B0E0F90180839183A283B38352
:10428000D9018D909D90AD90BC90F701C080D180F8
:10429000E280F380D8014D905D906D907C900E94FB
:1042A000D318FC014082518262827382C482D5821B
:1042B000E682F78280869186A286B386EF85F889AA
:1042C000E35CFD4FB081B983EF85F889EF5CFD4F6A
:1042D00080819181A281B3814F855889475B5D4F71
:1042E000FA01F081FB834F8558894E5A5D4FFA01E0
:1042F000F081FA834F8558894D5B5D4FFA01F0815B
:10430000FF834F8558894A5B5D4FFA01F081F8873A
:104310004F855889415B5D4FFA01F081F9874F85E0
:104320005889445B5D4FFA01F081FA87EF85F8897F
:10433000E25DFD4F2080EF85F889E151FE4F30802E
:10434000EF85F889EB5AFD4F40815181628173817D
:10435000EF85F889EE5DFD4F008111812281338167
:10436000EF85F889EA5EFD4FC080D180E280F3805E
:10437000EF85F889E65FFD4F80809180A280B38051
:10438000EF85F889EE50FE4F408051806280738047
:10439000EF85F88940A651A662A673A684A695A6C5
:1043A000A6A6B7A6C0AAD1AAE2AAF3AA04AB15ABE7
:1043B00026AB37AB40AF51AF62AF73AF34AE25AE73
:1043C0002A8525A3398536A34A8147A340E450E0D6
:1043D00060E070E0E05CFF4F408351836283738351
:1043E0002885EF85F88926AF3F8137AFAF014C5B59
:1043F0005F4F2B81FA012083EF85F889EB5BFF4F3C
:1044000080839183A283B383EF85F889E75BFF4FB5
:1044100039813083AF85B88955968D919C91569797
:104420008633910589F483EF94E2FD01E658FF4F4E
:104430009183808332961182108281EF94E23696C6
:1044400091838083329630C08C33910589F48BEE52
:1044500094E2EF85F889E658FF4F91838083EF85DA
:10446000F889E458FF4F1182108289EE94E212C05D
:104470008E97E1F483EE94E2EF85F889E658FF4FDA
:1044800091838083EF85F889E458FF4F1182108271
:104490008DED94E2EF85F889EE57FF4F918380838D
:1044A000EF85F889EC57FF4F11821082EF85F8896C
:1044B000838D948D4A97D1F48FEE94E2E258FF4FAA
:1044C00091838083EF85F889E058FF4F1182108235
:1044D0008DEE94E2EF85F889EA57FF4F9183808350
:1044E000EF85F889E857FF4F11821082EF85F88930
:1044F000E25CFD4F20812983EF85F889EB5CFD4F5D
:104500004080518062807380EF85F889E65BFD4FC3
:1045100030813B83EF85F889ED5AFD4F9081EF851F
:10452000F889EC5BFD4F40814F83EF85F889E95BAB
:10453000FD4F50815887EF85F889E05BFD4F808102
:10454000EF85F889E35BFD4FA081AA87EF85F889A5
:10455000E15DFD4F2080EF85F889E051FE4F30800E
:10456000EF85F889E75AFD4F2081318142815381DF
:104570002B873C874D875E87EF85F889EA5DFD4F85
:104580004081518162817381EF85F889E65EFD4F3C
:10459000C080D180E280F380EF85F889E25FFD4F33
:1045A00080809180A280B380EF85F889E657FF4F25
:1045B0002F8538892A503E4FD9010D911D912D919B
:1045C0003C91008F118F228F338F848E958EA68E13
:1045D000B78EC0A2D1A2E2A2F3A244A355A366A3C0
:1045E00077A32B853C854D855E8520A731A742A703
:1045F00053A734A625A63A85358B868B978B80E406
:1046000090E0A0E0B0E080AB91ABA2ABB3AB48854B
:1046100046A75F8157A78B8184AB45AA56AA67AA94
:1046200070AE998191AF858196818633910589F429
:1046300083EF94E2AF85B889AC50BF4F8D939C93C4
:10464000AF85B889AA50BF4F1D921C9281EF94E2AA
:1046500026C08C33910589F48BEE94E2AF85B8893E
:10466000AC50BF4F8D939C93AF85B889AA50BF4F74
:104670001D921C9289EE94E212C08E97E1F483EEB3
:1046800094E2AF85B889AC50BF4F8D939C93AF85B2
:10469000B889AA50BF4F1D921C928DED94E2AF8550
:1046A000B889A450BF4F8D939C93AF85B889A25011
:1046B000BF4F1D921C92838594854A97D9F48FEE43
:1046C00094E2EF85F889E850FF4F91838083EF856E
:1046D000F889E650FF4F118210828DEE94E2EF854B
:1046E000F889F39591838083EF85F889EE5FFE4F1B
:1046F00011821082EF85F889E15CFD4FA081A983CA
:104700002F853889275C3D4FD9018D919D910D9062
:10471000BC91A02D8B839C83AD83BE83EF85F889EC
:10472000E55BFD4FB081BA83EF85F889EC5AFD4F08
:1047300020812F83EF85F889EB5BFD4F308138872F
:10474000EF85F889E85BFD4F40814987EF85F8895F
:10475000EF5AFD4F2080EF85F889E25BFD4F3080F6
:10476000EF85F889E05DFD4F3081EF85F889EF50E6
:10477000FE4F2081EF85F889E35AFD4F80819181BA
:10478000A281B381EF85F889E65DFD4F40815181BB
:1047900062817381EF85F889E25EFD4FC080D18030
:1047A000E280F380EF85F889EE5EFD4F8080918096
:1047B000A280B3800F8518890C5F1E4FEF85F889A2
:1047C000E650FE4F4080518062807380F801408E39
:1047D000518E628E738E848E958EA68EB78EC0A2F9
:1047E000D1A2E2A2F3A244A355A366A377A380A714
:1047F00091A7A2A7B3A724A735A7358A268A2F8118
:10480000278B80E490E0A0E0B0E080AB91ABA2AB5E
:10481000B3AB298526A7388537A74A8144AB8B815E
:104820009C81AD81BE8185AB96ABA7ABB0AF298132
:1048300021AF858196818633910589F483EF94E2D7
:10484000EF85F889E259FE4F91838083EF85F889DF
:10485000E059FE4F1182108281EF94E226C08C3322
:10486000910589F48BEE94E2EF85F889E259FE4FC9
:1048700091838083EF85F889E059FE4F1182108281
:1048800089EE94E212C08E97E1F483EE94E2EF8514
:10489000F889E259FE4F91838083EF85F889E059CA
:1048A000FE4F118210828DED94E2EF85F889EA586F
:1048B000FE4F91838083EF85F889E858FE4F11827F
:1048C0001082D8011B968D919C911C974A97E1F418
:1048D0008FEE94E2EF85F889EE58FE4F9183808346
:1048E000EF85F889EC58FE4F118210828DEE94E22C
:1048F000EF85F889E658FE4F91838083EF85F8892C
:10490000E458FE4F11821082EF85F889E05CFD4F7C
:1049100020818F8598894096222311F0F2D101C021
:10492000DCD1EF85F889EF5BFD4F20818F85988979
:1049300086579F4F222311F0E4D101C0CED1EF85DD
:10494000F889EE5BFD4F80818823D1F0C801609625
:104950000FB6F894DEBF0FBECDBFDF91CF911F9190
:104960000F91FF90EF90DF90CF90BF90AF909F900E
:104970008F907F906F905F904F903F902F90C1C12C
:10498000C80160960FB6F894DEBF0FBECDBFDF91B1
:10499000CF911F910F91FF90EF90DF90CF90BF903C
:1049A000AF909F908F907F906F905F904F903F90CF
:1049B0002F9093C18FEF9FEF0895EBE0F1E080819E
:1049C000877F80830895EBE0F1E0808188608083B9
:1049D00008958E9808958E9A089514980895149ABB
:1049E000089588980895889A08950C94A3480C9483
:1049F000A3480C94A3480C94A3480C94A3480F9389
:104A00001F93CF93DF93FB0102A113A1C68DD78D16
:104A10000E94C432C530D105E1F064F4249771F5E9
:104A200064E070E08EED9CE00E94F710B8018EED1E
:104A30009CE022C0C630D105B1F02B97F9F46BE0B1
:104A400070E087EE9CE00E94F710B80187EE9CE0D2
:104A500013C065E070E081EE9CE00E94F710B801A1
:104A600081EE9CE009C066E070E084EE9CE00E946C
:104A7000F710B80184EE9CE00E94741080E090E092
:104A8000DF91CF911F910F9108958F929F92AF92D6
:104A9000BF92CF92DF92EF92FF920F931F930E94EB
:104AA00027171F921F9221E02F931F921F92812C94
:104AB000912CA12CB12CC12CD12C7601970186010F
:104AC000B701A6010E94D5020F900F900F900F9092
:104AD0000F9080E090E01F910F91FF90EF90DF909A
:104AE000CF90BF90AF909F908F9008950E94D31861
:104AF0000E94301880E090E0089560E0FC0183851A
:104B00000C94AB0E60E0FC0185810C94AB0E61E06F
:104B1000FC0183850C94AB0E61E0FC0185810C9453
:104B2000AB0ECF93DF93FB01C68DD78D0E9445322C
:104B3000BE010E94033280E090E0DF91CF910895A2
:104B4000CF93DF9380919F0B9091A00B892BF1F471
:104B50008CE390E00E940E48EC01FC01CC9611829F
:104B600010823C96E817F907D1F7198218821D8642
:104B70001C86198E188E1DA21CA219AA18AACE0175
:104B80000E94611BD093A00BC0939F0B80919F0B41
:104B90009091A00BDF91CF91089508950895089505
:104BA00008951F920F920FB60F9211240BB60F9219
:104BB0002F933F934F935F936F937F938F939F9325
:104BC000AF93BF93EF93FF93E0914207F0914307B8
:104BD0001995FF91EF91BF91AF919F918F917F9127
:104BE0006F915F914F913F912F910F900BBE0F905E
:104BF0000FBE0F901F901895CF93DF93EC01FC012F
:104C0000E759FF4F1082379781E0808360E08D8104
:104C10000E94AB0E8F859889892B31F060E08B85DF
:104C2000DF91CF910C94AB0EDF91CF910895CF938C
:104C3000DF93EC018B890E94830E2E8930E082176E
:104C4000930711F48F8901C080E0DF91CF9108951F
:104C5000CF93DF93EC0189890E94830E2E8930E087
:104C60008217930711F48F8901C080E0DF91CF9103
:104C70000895CF93DF93EC018DA5882311F061E0B7
:104C800001C060E08F810E94AB0E8EA5882329F0C1
:104C90008FA5882311F061E001C060E08D85DF9170
:104CA000CF910C94AB0ECF93DF93EC018DA58823AD
:104CB00011F060E001C061E08F810E94AB0E8EA513
:104CC000882329F08FA5882311F060E001C061E0FE
:104CD0008D85DF91CF910C94AB0ECF93DF93EC01D8
:104CE00061E089850E94AB0E8EA5882321F061E0EA
:104CF0008F850E94AB0EC959DF4F1882DF91CF918B
:104D00000895CF93DF93EC0160E089850E94AB0E9C
:104D10008EA5882321F060E08F850E94AB0EC959D3
:104D2000DF4F81E08883DF91CF910895CF92DF92AA
:104D3000EF92FF920F931F93CF93DF93FC0142AF4B
:104D400053AF64AF75AFDC01DE964D935D936D9309
:104D50007C93139714960D931D932D933C93139767
:104D6000EC01CA5BDF4FE88284A9882389F084A51F
:104D7000811109C037FF0CC01D921D921D921C921B
:104D8000139781E006C01016110612061306A4F34D
:104D900080E045A956A967A970AD14161506160638
:104DA00017063CF591AD992321F10D911D912D919F
:104DB0003C9113976801790137FF07C0CC24DD24AB
:104DC0007601C01AD10AE20AF30A4C155D056E0598
:104DD0007F057CF437FF07C070956095509541952D
:104DE0005F4F6F4F7F4F4D935D936D937C93139700
:104DF00081E0DF01A15BBF4F1D921D921D921C92AD
:104E00001397E15AFF4F91E09083DF91CF911F916B
:104E10000F91FF90EF90DF90CF9008950F931F9325
:104E2000CF93DF938C01D62FFC018589811109C0B6
:104E3000C8010EDFC82FC801FADED11108C08C2FBF
:104E400006C0C801F4DEC82FC80102DFF6CFDF912B
:104E5000CF911F910F910895CF93DF93EC01FC0147
:104E6000E759FF4F81E0808339978081B29788238B
:104E700041F080819181A281B3810196A11DB11D74
:104E800007C080819181A281B3810197A109B109F5
:104E900080839183A283B383FE01E459FF4F208175
:104EA0003181DE01A659BF4FC9019595879520FD37
:104EB00003C0ED91FC910DC0FE01E80FF91F0190B8
:104EC000F081E02D2D913C91E20FF31F0190F081D4
:104ED000E02D8C0F9D1F19958F859889892B11F1D5
:104EE000FE01E059FF4F20813181DE01A259BF4F01
:104EF000C9019595879520FD03C0ED91FC910DC0EA
:104F0000FE01E80FF91F0190F081E02D2D913C91F9
:104F1000E20FF31F0190F081E02D8C0F9D1FDF91B8
:104F2000CF911994DF91CF9108958F929F92AF9274
:104F3000BF92CF92DF92EF92FF920F931F93CF9386
:104F4000DF93EC01FC01E15BFF4F608171818281A5
:104F500093810E94B94D6B017C0168A979A98AA946
:104F60009BA90E94BB4D9B01AC0160E074E284E709
:104F700099E40E94A94F4B015C01FE01E55AFF4FE5
:104F800060817181828193810E94B94D9B01AC0146
:104F9000C501B4010E94A94F4B015C018E010D5A5D
:104FA0001F4F20E030E040E05FE30E941A4E9B017B
:104FB000AC01C701B6010E94454F0E941650F8018E
:104FC0006083718382839383C95ADF4FA501940163
:104FD000C701B6010E94454F0E941650688379832D
:104FE0008A839B83DF91CF911F910F91FF90EF9068
:104FF000DF90CF90BF90AF909F908F9008950F93C8
:105000001F93CF93DF93FC01E759FF4F20812223A9
:10501000B9F07A97008111812281338138964081DD
:10502000518162817381041715072607370710F134
:10503000EC01E2DDCE01DF91CF911F910F9175CF91
:10504000FC01E15AFF4F20812223A1F070970081DB
:105050001181228133813496408151816281738133
:10506000041715072607370728F0DF91CF911F9106
:105070000F91F2CEDF91CF911F910F9108952F9252
:105080003F924F925F926F927F928F929F92AF92D8
:10509000BF92CF92DF92EF92FF920F931F93CF9325
:1050A000DF93CDB7DEB762970FB6F894DEBF0FBEC1
:1050B000CDBF8C017C0126E4E20EF11CD7018C915E
:1050C0009801205A3F4FF801EF59FF4F6F01A80197
:1050D000425C5F4F4A0114971D01882341F0F8019B
:1050E00084A5D9018C9381E0F60180832FC0DA0179
:1050F0004D915D916D917C91F10180819181A281B1
:10510000B381BB24B394481759076A077B070CF097
:10511000B12CF901B08277FF07C07095609550956A
:1051200041955F4F6F4F7F4FB7FF07C0B095A09578
:10513000909581959F4FAF4FBF4F21E0481759077A
:105140006A077B070CF420E0D6012C93F401408120
:10515000518162817381411551056105710559F4D1
:10516000F801848D958DA68DB78DE55AFF4F80830C
:105170009183A283B383F10180819181A281B38164
:10518000F80142AC53AC64AC75AC9801215A3F4F66
:105190005901481659066A067B0634F44817590720
:1051A0006A077B077CF00AC084159505A605B7053C
:1051B0002CF484179507A607B70724F0D7018C9124
:1051C0008823D9F0F50180818823B9F0D7018C912B
:1051D000811105C0F701808181110FC006C060E018
:1051E000C8011CDE8111F6CF17C0D6016C9181E099
:1051F0006827C80113DE882379F0D5011C9260E08E
:10520000C8010CDE882309F4C6C1F801FE9610829D
:10521000118212821382BFC1D80194962D913D91C3
:105220004D915C91979729833A834B835C83589681
:105230002D913D914D915C915B972D833E834F83E2
:1052400058875C962D913D914D915C915F97298790
:105250003A874B875C87F10180819181A281B3817C
:10526000F801FE96C080D180E280F380F80142AD63
:1052700053AD64AD75ADED59FF4F1082319610827C
:105280003801F5E66F0E711CF301108298012A595E
:105290003F4FF9011082329610824C015D01841A51
:1052A000950AA60AB70AB7FE08C0B094A0949094D5
:1052B0008094811C911CA11CB11C481759076A07D6
:1052C0007B072CF4C41AD50AE60AF70A04C0C81AE8
:1052D000D90AEA0AFB0AD501C401B595A7959795A5
:1052E00087958D879E87AF87B88BD801A859BF4F08
:1052F0001D01F7FC05C08C149D04AE04BF044CF4E2
:10530000F80100A0F1A1E02DFA8BE98B81E0D90131
:105310001BC02D853E854F8558892C153D054E05B2
:105320005F0508F454C089819A81AB81BC818C15DA
:105330009D05AE05BF0564F42D813E812F5F3F4F73
:105340003A8B298B81E0D3018C93F10180839EC03D
:10535000C701B6010E94BB4D2B013C0169817A81D6
:105360008B819C810E94BB4D9B01AC01C301B201AA
:105370000E94A94F2B013C016D817E818F81988510
:1053800029853A854B855C85621B730B840B950BD5
:105390000E94BB4D9B01AC01C301B2010E941A4E99
:1053A0002B013C0169857A858B859C850E94BB4DCC
:1053B0009B01AC01C301B2010E94454F0E941150F4
:1053C0007A8B698B81E0F801ED59FF4F5CC0D50104
:1053D000C40129813A814B815C81821B930BA40B10
:1053E000B50BC816D906EA06FB065CF42D813E8192
:1053F0002E5F3F4F3A8B298B81E0F801EB59FF4F2D
:1054000042C0C501B4016C197D098E099F090E9433
:10541000BB4D2B013C0169817A818B819C810E946B
:10542000BB4D9B01AC01C301B2010E94A94F2B01EE
:105430003C016D817E818F81988529853A854B85D8
:105440005C85621B730B840B950B0E94BB4D9B010B
:10545000AC01C301B2010E941A4E2B013C016985C7
:105460007A858B859C850E94BB4D9B01AC01C30155
:10547000B2010E94454F0E9411507A8B698B81E0E6
:10548000F801EC59FF4F8083D1018C93F80184819E
:105490008823B1F00E941E10D80112964D905C90A6
:1054A0001397052C000C66087708DC01CB018419E2
:1054B0009509A609B709893E9340A105B10568F48D
:1054C000F801E55AFF4F29893A89C901A0E0B0E007
:1054D00080839183A283B38392CE0E941E10D80151
:1054E00013967C936E93129784E294E00E94E33BC0
:1054F00081EB95E00E94E33B60E070E0CB010E940D
:105500002F3C87EB95E00E94E33BC701B6010E9468
:105510002F3C8DEB95E00E94E33BC501B4010E9456
:105520002F3C83EC95E00E94E33B4AE06D857E854D
:105530008F8598890E94E43B8AEC95E00E94E33BCA
:1055400069817A818B819C810E942F3C80ED95E05E
:105550000E94E33B69857A858B859C850E942F3C60
:1055600086ED95E00E94E33B6D817E818F81988579
:105570000E942F3C8CED95E00E94E33B8EE496E088
:105580000E94E33B89899A890E94563C8CE993E00A
:105590000E94E33B95CF62960FB6F894DEBF0FBE34
:1055A000CDBFDF91CF911F910F91FF90EF90DF90D2
:1055B000CF90BF90AF909F908F907F906F905F90B3
:1055C0004F903F902F9008950F931F93FC01EA5B3B
:1055D000FF4F2081211110C0389700811181228155
:1055E000338134964081518162817381041715079C
:1055F0002607370744F404C0FC0124A5222319F030
:105600001F910F9150CB1F910F9133CBFC0113824F
:1056100012821482168215821086178212861186D3
:105620001486138616861586108A1786128A118AA2
:10563000148A138ADC01A15ABF4F1C9212AE13AE1A
:1056400014AE15AE91971D921D921D921C92139748
:1056500014961D921D921D921C92139714961C92E3
:105660005A961C9211961C9212961C9211961C929C
:1056700011961C9211961C9211961C9211961C92D6
:1056800011961C9211968CE895E211969C938E933C
:10569000129611961C921E92129687E895E2119628
:1056A0009C938E93129611961C921E92129682E8EB
:1056B00095E211969C938E93129611961C921E92CF
:1056C00012968DE795E28D939C93E858FF4F1182D7
:1056D0001082089508956E3471050CF050C06B343B
:1056E00071050CF08FC06C32710554F5693271058B
:1056F0000CF088C06831710594F46F3071050CF0BE
:1057000081C06630710544F4623071050CF07AC0D6
:10571000672B09F075C076C06B5071096EC062329C
:1057200071053CF46F3171050CF06CC06951710961
:1057300064C0645271096230710508F061C062C0D2
:105740006A3371057CF4673371050CF05BC06D3210
:1057500071050CF455C0603371050CF453C06353EC
:1057600071094BC0643471053CF4613471050CF06F
:1057700049C06D53710941C0675471093EC0663814
:105780007105F4F463387105ECF56237710564F462
:105790006F367105BCF56536710594F16836710593
:1057A0008CF16956710929C06C37710534F4693779
:1057B000710544F56357710920C06D5771091DC00B
:1057C000603D71057CF46D3C7105E4F4643971054C
:1057D00034F461397105B4F46D5871090EC0695C17
:1057E00071090BC06A3D710534F4673D710554F4CD
:1057F000635D710902C06D5D71096330710510F060
:1058000080E0089581E00895603E710508F0D8C3F6
:10581000FB018827EC57FF4F8F4F0C94655081E0B8
:1058200090E0A0E0B0E08093560790935707A093D4
:105830005807B0935907089510925A0710925B07C2
:1058400010925C0710925D07089510925E07109207
:105850005F071092600710926107089581E090E061
:10586000A0E0B0E08093620790936307A093640781
:10587000B09365070895109266071092670710921B
:10588000680710926907089583E090E0A0E0B0E017
:1058900080936A0790936B07A0936C07B0936D0792
:1058A000089588E790E0A0E0B0E0809382079093AD
:1058B0008307A0938407B0938507089588E790E055
:1058C000A0E0B0E08093860790938707A0938807B5
:1058D000B0938907089588E790E0A0E0B0E0809356
:1058E0008A0790938B07A0938C07B0938D07089538
:1058F00010929207109293071092940710929507B6
:105900000895109296071092970710929807109298
:105910009907089581E090E0A0E0B0E080939A07B5
:1059200090939B07A0939C07B0939D0708951092B6
:105930009E0710929F071092A0071092A10708954A
:105940001092A2071092A3071092A4071092A50725
:1059500008951092A6071092A7071092A807109218
:10596000A90708951092AA071092AB071092AC07EE
:105970001092AD0708951092AE071092AF071092E3
:10598000B0071092B10708951092B2071092B307B2
:105990001092B4071092B50708951092BA071092AA
:1059A000BB071092BC071092BD0708951092BE0766
:1059B0001092BF071092C0071092C107089510926D
:1059C000C2071092C3071092C4071092C50708952A
:1059D0001092D2071092D3071092D4071092D507D5
:1059E00008951092D6071092D7071092D8071092F8
:1059F000D90708951092DA071092DB071092DC079E
:105A00001092DD07089581E090E0A0E0B0E080937F
:105A1000E6079093E707A093E807B093E907089596
:105A200081E090E0A0E0B0E08093EA079093EB077C
:105A3000A093EC07B093ED0708958CE291E0A0E00D
:105A4000B0E08093FA079093FB07A093FC07B09314
:105A5000FD0708958CE291E0A0E0B0E08093FE079E
:105A60009093FF07A0930008B093010808958CE27B
:105A700091E0A0E0B0E08093020890930308A09327
:105A80000408B0930508089510920A0810920B08B4
:105A900010920C0810920D08089510920E081092A2
:105AA0000F08109210081092110808951092120811
:105AB000109213081092140810921508089510926D
:105AC00022081092230810922408109225080895A5
:105AD0001092260810922708109228081092290880
:105AE000089581E090E0A0E0B0E080932A089093D0
:105AF0002B08A0932C08B0932D08089585E090E022
:105B0000A0E0B0E08093320890933308A09334086B
:105B1000B0933508089585E090E0A0E0B0E0809370
:105B2000360890933708A0933808B0933908089541
:105B300089E190E0A0E0B0E080933A0890933B08C0
:105B4000A0933C08B0933D08089582E390E0A0E064
:105B5000B0E080934A0890934B08A0934C08B09310
:105B60004D08089582E390E0A0E0B0E080934E08F5
:105B700090934F08A0935008B0935108089582E382
:105B800090E0A0E0B0E08093520890935308A09377
:105B90005408B0935508089582E390E0A0E0B0E087
:105BA00080935A0890935B08A0935C08B0935D08BB
:105BB000089582E390E0A0E0B0E080935E089093C7
:105BC0005F08A0936008B0936108089582E390E0B5
:105BD000A0E0B0E08093620890936308A09364080B
:105BE000B0936508089580E991E0A0E0B0E080936B
:105BF000720890937308A0937408B0937508089581
:105C000080E991E0A0E0B0E0809376089093770877
:105C1000A0937808B0937908089580E991E0A0E016
:105C2000B0E080937A0890937B08A0937C08B093AF
:105C30007D080895109282081092830810928408BB
:105C40001092850808951092860810928708109285
:105C5000880810928908089510928A0810928B087B
:105C600010928C0810928D08089510929A09109243
:105C70009B0910929C0910929D09089510929E090B
:105C800010929F091092A0091092A10908951092F4
:105C9000A2091092A3091092A4091092A5090895CF
:105CA0001092EA081092EB081092EC081092ED089E
:105CB00008951092EE081092EF081092F0081092DA
:105CC000F10808951092F2081092F3081092F40867
:105CD0001092F50808951092FA081092FB0810929D
:105CE000FC081092FD0808951092FE081092FF081B
:105CF0001092000910920109089510920209109261
:105D000003091092040910920509089585E090E0B6
:105D1000A0E0B0E08093120990931309A0931409B6
:105D2000B0931509089585E090E0A0E0B0E080937D
:105D3000160990931709A0931809B09319090895AB
:105D400085E090E0A0E0B0E080931A0990931B09F1
:105D5000A0931C09B0931D09089584EB95E1A0E080
:105D6000B0E08093220990932309A0932409B09373
:105D70002509089584EB95E1A0E0B0E08093260921
:105D800090932709A0932809B0932909089584EBDB
:105D900095E1A0E0B0E080932A0990932B09A093AD
:105DA0002C09B0932D09089585E090E0A0E0B0E0C3
:105DB00080933A0990933B09A0933C09B0933D0925
:105DC000089585E090E0A0E0B0E080933E099093D4
:105DD0003F09A0934009B0934109089585E090E000
:105DE000A0E0B0E08093420990934309A093440956
:105DF000B0934509089510924A0910924B091092E8
:105E00004C0910924D09089510924E0910924F09B5
:105E1000109250091092510908951092520910924F
:105E2000530910925409109255090895109262096D
:105E300010926309109264091092650908951092F6
:105E4000660910926709109268091092690908950D
:105E500010926A0910926B0910926C0910926D09E8
:105E6000089510927A0A10927B0A10927C0A10927E
:105E70007D0A08958CE390E0A0E0B0E080937E0A74
:105E800090937F0AA093800AB093810A089581E0DD
:105E900090E0A0E0B0E08093820A9093830AA09300
:105EA000840AB093850A089510928A0A10928B0A88
:105EB00010928C0A10928D0A08958CE390E0A0E075
:105EC000B0E080938E0A90938F0AA093900AB093CB
:105ED000910A089581E090E0A0E0B0E08093920AFA
:105EE0009093930AA093940AB093950A0895109200
:105EF000A20A1092A30A1092A40A1092A50A089569
:105F00008CE390E0A0E0B0E08093A60A9093A70A0B
:105F1000A093A80AB093A90A089581E090E0A0E0B8
:105F2000B0E08093AA0A9093AB0AA093AC0AB09316
:105F3000AD0A08951092B20A1092B30A1092B40AF0
:105F40001092B50A08958CE390E0A0E0B0E0809351
:105F5000B60A9093B70AA093B80AB093B90A089505
:105F600081E090E0A0E0B0E08093BA0A9093BB0A91
:105F7000A093BC0AB093BD0A08951092CA0A109269
:105F8000CB0A1092CC0A1092CD0A08958CE390E0CF
:105F9000A0E0B0E08093CE0A9093CF0AA093D00AFD
:105FA000B093D10A089581E090E0A0E0B0E0809342
:105FB000D20A9093D30AA093D40AB093D50A089535
:105FC000660F771F660F771FFB01EA5AF84F1082A2
:105FD00011821282138208950F931F93CF93DF9340
:105FE0008C01C0E0D0E0BE01C80175DB882319F048
:105FF000BE01C80109DC2196C13ED105A1F7DF91A0
:10600000CF911F910F9108954F925F926F927F925F
:106010008F929F92AF92BF92CF92DF92EF92FF92B8
:10602000CF93DF935B01EB01CC0FDD1FCE010E940C
:10603000D14E482E512C612C712CCE0101960E941C
:10604000D14EC82ED12CE12CF12C8DE8A81AB10824
:1060500083E0A816B10488F5CE0144960E94D14E83
:10606000882E912CA12CB12CCE0145960E94D14EA8
:10607000482F50E060E070E08FEF88169104A10493
:10608000B104A9F44F3F51056105710581F48FEF0B
:10609000481651046104710481F48FEFC816D104CD
:1060A000E104F10451F46FEF7FEFCB012BC04038D6
:1060B0005105610571056CF0F6CF80E8C816D10472
:1060C000E104F10484F740E050E0BA01812C912C06
:1060D0005401FE2CED2CDC2CCC24C40CD51CE61C6D
:1060E000F71C540199248824C80CD91CEA1CFB1CF9
:1060F000742F662755274427CB01BA016C0D7D1DEF
:106100008E1D9F1DDF91CF91FF90EF90DF90CF907C
:10611000BF90AF909F908F907F906F905F904F90C7
:1061200008950C94A3480C94A3480C94A348CF93CF
:10613000DF93EB0120E030E040E85FE36A817B81A0
:106140008C819D810E94B54D811113C082EE95E036
:106150000E94E33B0E942717FC01E25BFF4F108285
:10616000118212821382E05DFE4F108A118A128A18
:10617000138A20E030E040E85FE36E817F8188850C
:1061800099850E94B54D811113C082EF95E00E9460
:10619000E33B0E942717FC01E853FF4F1082118256
:1061A00012821382EC52FF4F108A118A128A138ACC
:1061B00020E030E040E85FE36A857B858C859D8543
:1061C0000E94B54D811113C082E096E00E94E33B2E
:1061D0000E942717FC01EE5BFE4F10821182128293
:1061E0001382E858FF4F108A118A128A138A0E947C
:1061F000D3180E94DD1780E090E0DF91CF910895E1
:106200000F93CF93DF938091A30B811178C081E02E
:106210008093A30B0E942717EC0103B123B1409197
:10622000000160910001001F0027001F221F22278C
:10623000221F41706695617082589E4F29D503B127
:1062400023B140B160B1001F0027001F221F222789
:10625000221F42FB442740F966956170CE018456A7
:106260009E4F16D503B123B140B160B1001F002786
:10627000001F221F2227221F46FB442740F9661FCA
:106280006627661FCE0186549E4F02D5FE01E15956
:10629000FF4F8081882361F0709780819181A28176
:1062A000B3810196A11DB11D80839183A283B38325
:1062B000FE01E751FF4F8081882361F07097808154
:1062C0009181A281B3810196A11DB11D808391832B
:1062D000A283B383FE01ED59FE4F8081882369F0CC
:1062E000CD5ADE4F88819981AA81BB810196A11D7B
:1062F000B11D88839983AA83BB831092A30BDF917E
:10630000CF910F9108958F929F92AF92BF92CF92AB
:10631000DF92EF92FF920F931F930E94271721E0C5
:106320002F931F921F921F921F92812C912CA12CB0
:10633000B12CC12CD12C760197018601B701A601A1
:106340000E94D5020F900F900F900F900F9080E059
:1063500090E01F910F91FF90EF90DF90CF90BF9052
:10636000AF909F908F900895EF92FF920F931F939D
:10637000CF93DF9300D01F92CDB7DEB78B017B01A7
:10638000EE0CFF1C622FC70129833A834B835C8389
:106390000E94D94E29813A814B815C81992757FD12
:1063A0009A95852F742F632FC70101960E94D94EAD
:1063B0000D58110929813A814B815C810330110507
:1063C000A8F4BA01992777FD9095892FC7014496C3
:1063D0000E94D94E29813A814B815C81652F7727B4
:1063E00088279927C70145960E94D94E80E090E002
:1063F0000F900F900F900F90DF91CF911F910F9101
:10640000FF90EF900895CF92DF92EF92FF92CF939B
:10641000DF93EB0160D9882359F1FE01EE0FFF1FD6
:10642000EE0FFF1FEA5AF84FC080D180E280F38060
:1064300082E196E00E94E33B8EE496E00E94E33B1B
:1064400086E196E00E94E33BCE010E94563C8EE43A
:1064500096E00E94E33B88E196E00E94E33BC7019F
:10646000B6010E942F3C0E94D3180E94DD1704C081
:106470008AE196E00E94E33B80E090E0DF91CF91DB
:10648000FF90EF90DF90CF900895EF92FF920F93DF
:106490001F93CF93DF938091A40B9091A50B892B31
:1064A00009F064C084E090E00E940E48EC0160E0D6
:1064B00070E0AADD16161706F4F0CE018DDD96E524
:1064C000E92E97E0F92E00E010E0B801CE0103D9E3
:1064D000882341F0F7012081318142815381B80145
:1064E000CE0142DF0F5F1F4FF4E0EF0EF11C0639C3
:1064F000110559F737C063E070E0CE0185DD6130EA
:1065000071058105910561F586E5E82E87E0F82E95
:1065100000E010E0B801CE01DED88823C1F0B80158
:10652000CE0172DDF70160837183828393836F3FB5
:106530007F4F8F4F9F4F59F4B801CE0165D9F701B6
:106540002081318142815381B801CE010DDF0F5F7F
:106550001F4FF4E0EF0EF11C013E1105D9F602C009
:10656000CE013ADDD093A50BC093A40B8091A40B70
:106570009091A50BDF91CF911F910F91FF90EF901C
:1065800008950895089508958091A10B9091A20B0C
:10659000892B41F481E090E00E940E489093A20B79
:1065A0008093A10B8091A10B9091A20B0895EF9283
:1065B000FF920F931F93CF93DF93162F072F7A012C
:1065C0004115510559F4862F0E94830E31E020E0D9
:1065D000019709F030E0C32FD22F26C0413051057A
:1065E00009F5262F663310F02AEC260F80917B00E8
:1065F000922F9870877F892B80937B00277020646F
:1066000020937C0080917A00806480937A0080914E
:106610007A0086FDFCCFC091780080917900D0E0AF
:10662000D82B02C0C0E0D0E082E0E816F10410F5FB
:106630008CE396E00E94E33B8EE496E00E94E33B0D
:1066400086E196E00E94E33B812F902F0E94563C0A
:106650008EE496E00E94E33B88E196E00E94E33BF3
:10666000CE010E94563C0E94D3180E94DD1780E0A4
:1066700090E002C081E090E0DF91CF911F910F91F7
:10668000FF90EF90089580E496E00E94E33B0E9423
:10669000D3180E941A1B0E94D3180E94EF171DD214
:1066A00040E050E068E070E082DF17D240E050E068
:1066B00069E070E07CDF11D240E050E06AE070E019
:1066C00076DF0BD240E050E06DE070E070DF80E0FC
:1066D00090E008950F931F93CF93DF938B01EA010E
:1066E000AB01415051094433510508F0D4C0223068
:1066F000310508F0D0C048E3429FF001439FF00D00
:106700001124E60FF71FE80FF91F81E08083232B88
:1067100011F46C2F07C061E0802F0E949F0F20971B
:1067200039F460E0802F0E94AB0E80E090E0B5C0AD
:10673000CF3FD10509F4ADC0F801EF5DFB4FE49107
:106740008E2F90E0FC013197E231F10508F09DC0F9
:106750008827EC59FE4F8F4F0C94655084B58068A4
:1067600084BDC7BDE2CF84B5806284BDC8BDDDCF26
:1067700080918000806880938000D0938900C093CE
:106780008800D3CF80918000806280938000D09376
:106790008B00C0938A00C9CF80918000886080936D
:1067A0008000D0938D00C0938C00BFCF8091B0004B
:1067B00080688093B000C093B300B7CF8091B000E1
:1067C00080628093B000C093B400AFCF80919000FE
:1067D000806880939000D0939900C0939800A5CFD3
:1067E00080919000806280939000D0939B00C09332
:1067F0009A009BCF80919000886080939000D09306
:106800009D00C0939C0091CF8091A00080688093F0
:10681000A0008091A0008F7B8093A000D093A9005E
:10682000C093A80082CF8091A00080628093A000D6
:10683000D093AB00C093AA0078CF8091A00088606D
:106840008093A000D093AD00C093AC006ECF809138
:106850002001806880932001D0932901C0932801F2
:1068600064CF80912001806280932001D0932B011E
:10687000C0932A015ACF8091200188608093200123
:10688000D0932D01C0932C0150CFC038D1050CF40A
:1068900048CF61E047CF81E090E0DF91CF911F9139
:1068A0000F9108950C94A3480C94A3480C94A3480A
:1068B0000C94A3480C94A3480C94A3480C94A348AC
:1068C0000C94A3480C94A3480C94A3480C94A3489C
:1068D0008F929F92AF92BF92CF92DF92EF92FF92F0
:1068E0000F931F930E94271760E070E04ED2892B10
:1068F000D1F40E9427171F921F9221E02F931F921D
:106900001F92812C912CA12CB12CC12CD12C760161
:1069100097018601B701A6010E94D5020F900F9042
:106920000F900F900F9080E090E01F910F91FF90DB
:10693000EF90DF90CF90BF90AF909F908F90089591
:106940008F929F92AF92BF92CF92DF92EF92FF927F
:106950000F931F930E94271761E070E016D2892BD6
:10696000D1F40E9427171F9221E02F931F921F92AC
:106970001F92812C912CA12CB12CC12CD12C7601F1
:1069800097018601B701A6010E94D5020F900F90D2
:106990000F900F900F9080E090E01F910F91FF906B
:1069A000EF90DF90CF90BF90AF909F908F90089521
:1069B000EF92FF920F931F93CF93DF9300D01F921C
:1069C000CDB7DEB7FB0122A133A144A155A1068DAD
:1069D000178D29833A834B835C8357DD7C01FC014F
:1069E0008281938129813A814B815C818F30F7E2EA
:1069F0009F072CF40196F7019383828303C0F7016C
:106A000013821282B801C70129833A834B835C83C6
:106A10000E946B2B29813A814B815C81882391F004
:106A2000F801EE0FFF1FEE0FFF1FEA5AF84F208309
:106A3000318342835383B801C70196DCB801C70193
:106A4000E2DC03C08AE196E0BED60E94A0250E9447
:106A5000611B80E090E00F900F900F900F90DF91FE
:106A6000CF911F910F91FF90EF9008950F931F9377
:106A7000CF93DF930ADD8C01C0E0D0E0BE01C801F6
:106A80000E946B2B882319F0BE01C801BCDC219643
:106A9000C13ED10599F787E496E095D60E94D318B8
:106AA0000E94DD1780E090E0DF91CF911F910F9160
:106AB00008958BE496E087D685E593E084D60E941E
:106AC000D3180E94DD1780E090E008950E94D3184B
:106AD000FC01148680E090E008958091A60B9091CF
:106AE000A70B892BA1F480E790E00E940E48FC01DF
:106AF000F9969C0123593F4FDF01D8971C921192C0
:106B0000E217F307C9F79093A70B8093A60B809128
:106B1000A60B9091A70B08956F927F928F929F92F0
:106B2000AF92BF92CF92DF92EF92FF920F931F939B
:106B3000CF93DF93FB01E2A8F3A886A497A4A0A8B3
:106B4000B1A8C6A0D7A062A073A0068D178DC5DF1F
:106B5000EC019701A301B801BDDDC501B4010E949C
:106B6000E60F9701A601B801CE01B4DD80E090E008
:106B7000DF91CF911F910F91FF90EF90DF90CF9019
:106B8000BF90AF909F908F907F906F9008950F93DC
:106B90001F93CF93DF93FB0102A913A9C68DD78D55
:106BA0009CDFA801BE0103DD80E090E0DF91CF9182
:106BB0001F910F9108951F93CF93DF931F92CDB72D
:106BC000DEB7FB0162A9168D698387DF6981812F9A
:106BD0000E949F0F80E090E00F90DF91CF911F9176
:106BE0000895EF92FF920F931F93CF93DF93FB01D2
:106BF000E2A8F3A802A113A1C68DD78D6EDF97017D
:106C0000A801BE0167DD80E090E0DF91CF911F9188
:106C10000F91FF90EF9008950895089508950895B5
:106C20000895CF93DF93EC0188810E94830E21E0C9
:106C3000892B09F420E02C878C810E94830E21E0AF
:106C4000892B09F420E02E87888D998D0197D1F446
:106C50008A810E94830E21E0892B09F420E02D8790
:106C60008E810E94830E21E0892B09F420E02F877A
:106C70009C858D85981749F08E85821731F09A870B
:106C80008B8703C08C858A872B87DF91CF910895EE
:106C90000F93FC019285908783858187A08DB18DAC
:106CA000119721F4621721F0401711F06287438792
:106CB00083858823D1F0828591110AC08823A9F0A9
:106CC00080899189A289B3890197A109B10909C075
:106CD00081110BC080899189A289B3890196A11D78
:106CE000B11D808B918BA28BB38B0F910895CF93A5
:106CF000DF93FC012489358946895789C28DD38D5C
:106D000060897189828993892031E7E23E074105D4
:106D1000510529F0121613061406150624F0DE019B
:106D20009B01AC0109C00E944A5020E137E240E0DB
:106D300050E00E94E74EDE010E940D4FDF91CF919F
:106D40000895FC0181E090E0958F848F118210827C
:106D500015821482108A118A128A138A118E108E5B
:106D600080E197E2A0E0B0E0848B958BA68BB78B97
:106D7000128610861486158616861786089508953D
:106D8000089508950895089508952F923F924F927F
:106D90005F926F927F928F929F92AF92BF92CF92AB
:106DA000DF92EF92FF920F931F93CF93DF93CDB7B4
:106DB000DEB7A3970FB6F894DEBF0FBECDBF9BA37F
:106DC0008AA31B010E94831D8AA19BA10E94961B7E
:106DD0008AA19BA10E9487138AA19BA10E9489136B
:106DE00021E022163104C9F132E02316310409F4FE
:106DF00066C02114310409F095C0AAA0BBA040E1EF
:106E0000A40EB11C8AA19BA182589E4F9E838D83A4
:106E1000EAA1FBA1E45BFD4F90819B87AAA1BBA1E6
:106E2000A359BD4FB887AF83EAA1FBA1E956FD4F37
:106E3000FF87EE872AA13BA127553D4F3B8B2A8B2D
:106E40004AA15BA147515E4F5A8749878DE890E080
:106E5000998B888BA5E1B0E062C0AAA0BBA0BAE87C
:106E6000AB0EB11CEAA1FBA1E456FE4FFE83ED83FD
:106E7000EAA1FBA1E35BFD4F20812B874AA15BA127
:106E80004F585D4F58874F838AA19BA187569D4FCE
:106E90009F878E87AAA1BBA1A655BD4FBB8BAA8B8E
:106EA000EAA1FBA1E551FE4FFA87E9872EE830E021
:106EB000398B288B46E150E05C834B8336C0AAA017
:106EC000BBA05CEFA51A5EEFB50A8AA19BA1865410
:106ED0009E4F9E838D83EAA1FBA1E25BFD4F9081D3
:106EE0009B87AAA1BBA1AB58BD4FB887AF83EAA1CE
:106EF000FBA1E556FD4FFF87EE872AA13BA1255553
:106F00003D4F3B8B2A8B4AA15BA143515E4F5A8771
:106F100049878FE890E0998B888BA7E1B0E0BC832C
:106F2000AB8303C080E596E00CC0C5010E94282613
:106F3000811105C0C5010E941726882369F081EEE2
:106F400096E041D40E94D31881E090E090934507E9
:106F50008093440790E0D4C384E294E034D48FE774
:106F600096E031D4D5018C916FD487E197E02BD492
:106F70008CE993E028D481E090E0E985FA8591835B
:106F8000808341E050E0B5018AA19BA10E942B19AA
:106F9000C5010E948126D5019C968C918501005ADD
:106FA0001F4F882339F0C5010E94532681E0F80164
:106FB000808305C0C5010E943926D8011C928D81AD
:106FC0009E8195DEF501FE966083718382839383B3
:106FD000EF81F8851082118212821382EAA1FBA14F
:106FE000E359FD4F1082118212821382EAA1FBA1A4
:106FF000EF58FD4F1082118212821382EAA1FBA189
:10700000EB58FD4F108211821282138286E090E0CD
:10701000A985BA858D939C9346E050E0B5018AA17D
:107020009BA10E942B1941E050E0B5018AA19BA1D0
:107030000E941019412C512C320143948AA19BA12A
:10704000820D931DFC01E755FD4FFD87EC87410143
:10705000880C991C880C991CC40183569D4F2AA149
:107060003BA1280F391F3D8B2C8BC101815A9E4FAC
:10707000880F991F4AA15BA1480F591F598F488F4C
:10708000C40185579D4FAAA1BBA1A80FB91FBB8FF3
:10709000AA8FF401E158FD4FFD8FEC8F8AA19BA1CF
:1070A000880D991D9C012A5E3D4F3F8F2E8FAC8528
:1070B000BD858C918823B1F0A40143595D4FEAA1AD
:1070C000FBA14E0F5F1FCC88DD88E88CF98C0A8D00
:1070D0001B8D2C8D3D8D2E0F3F1F6D817E81C50137
:1070E0000E94CB1288EA9BE00E948E0B18161906AC
:1070F00024F01A82198210E01DC088EA9BE00E94E9
:107100006C0B8F7D85349105A1F78DE994E05BD3FD
:107110000E94D31821E0DC011C962C9382E693E0B8
:1071200052D30E94D3180E94DD17E1E0F0E0FA8309
:10713000E98311E0C5010E9428268111D0C2C50152
:107140000E9417268111CBC21111C9C2AE85BF851D
:107150006D917C91072E000C880B990B0E94BB4D02
:107160009B01AC01EF81F8856081718182819381FF
:107170000E94B54D87FFB3C2C5010E942C278AA18A
:107180009BA1880D991D8C010A5E1D4FF80120817D
:1071900031814281538160E573EC80E090E00E9490
:1071A000E74EC9010E94DB0FD8012D913D914D9111
:1071B0005C91A3E0B0E00E94034F9B01AC01C301CE
:1071C000B2010E94E74E672B682B692B39F48EE5DC
:1071D00093E0F9D20E94D3180E94DD17C5010E94E6
:1071E000FC25AE8DBF8D2D913D914D915C9160E55B
:1071F00073EC80E090E00E94E74EC9010E94DB0F33
:10720000BFEF4B1A5B0A6B0A7B0AE981FA81EF2B0D
:1072100009F44DCF21E030E03A83298342E050E089
:10722000B5018AA19BA10E94101984E294E0CBD2FF
:107230008FE796E0C8D2D5018C9106D386E896E018
:10724000C2D28CE993E0BFD2E981FA81EF2BD1F46D
:1072500089E996E0B8D28EE496E0B5D286E196E070
:10726000B2D28B819C8122D38EE496E0ACD288E1AD
:1072700096E0A9D2FB858F2F90E018D30E94D318F7
:107280000E94DD178AA19BA10E9487138AA19BA15E
:107290000E94891384E294E096D28FE796E093D21D
:1072A000D5018C91D1D28DE996E08DD28CE993E015
:1072B0008AD2EF81F8851082118212821382D50161
:1072C0009C968C918501005A1F4F882331F0C5018F
:1072D0000E943926F801108206C0C5010E9453267B
:1072E00081E0D8018C938D819E8101DDF501FE96B0
:1072F0006083718382839383EAA1FBA1E359FD4FED
:107300001082118212821382EAA1FBA1EF58FD4F75
:107310001082118212821382EAA1FBA1EB58FD4F69
:1073200010821182128213828D819E81E0DC6C8B2F
:107330007D8B8E8B9F8B412C512C320143948AA1E3
:107340009BA1820D931DFC01E755FD4FF98FE88F3E
:107350009101220F331F220F331F3C832B83C9015E
:1073600083569D4F4AA15BA1480F591F5B8F4A8FDF
:10737000C101815A9E4F880F991FAAA1BBA1A80FD6
:10738000B91FBD8FAC8FC90185579D4FEAA1FBA1E5
:10739000E80FF91FFF8FEE8FC9012AA13BA1820FD1
:1073A000931FAC014A5E5D4F59A348A3F201319788
:1073B000FD87EC874F0129813A81232B09F0CFC04B
:1073C000A88DB98D8C918823C9F02B813C812158DF
:1073D0003D4FEAA1FBA12E0F3F1F4B815C8143591A
:1073E0005D4F4E0F5F1FCA8CDB8CEC8CFD8C0E8DBD
:1073F0001F8D6D817E81C5010E94CB1288EA9BE0C2
:107400000E948E0B1816190614F010E01DC088EAB1
:107410009BE00E946C0B8F7D85349105B1F78DE95F
:1074200094E0D1D10E94D31821E0DC011C962C936A
:1074300082E693E0C8D10E94D3180E94DD17E1E0F4
:10744000F0E0FA83E98311E02C853D852A3031058F
:1074500038F4AF81B8851D921D921D921C9213972E
:10746000BB85C501B11147C10E941726811173C0A8
:10747000112319F08C849D846EC0EE85FF85608198
:107480007181072E000C880B990B0E94BB4D9B014C
:10749000AC01AF81B8856D917D918D919C910E94D9
:1074A000B54D87FFE7CFC5010E942C278B809C80BC
:1074B000EAA1FBA18E0E9F1EFAEE8F1AFDEF9F0A26
:1074C000D4012D913D914D915C9160E573EC80E08C
:1074D00090E00E94E74EC9010E94DB0FF401208179
:1074E000318142815381A3E0B0E00E94034F9B01B0
:1074F000AC01C301B2010E94E74E672B682B692BD8
:1075000091F48EE593E05FD10E94D3180E94DD17BD
:1075100084E294E058D181EB96E055D1C201C6D106
:107520008CE993E050D1C5010E94FC25A8A1B9A126
:107530002D913D914D915C9160E573EC80E090E080
:107540000E94E74EC9010E94DB0FBFEF4B1A5B0A96
:107550006B0A7B0A2BCF8FEB96E035D104C041E05C
:1075600050E05A83498384E294E02DD18FE796E07E
:107570002AD1D5018C9168D183ED96E024D18CE994
:1075800093E021D18D819E81B2DBEA89FB89EF2BCB
:10759000A1F0DC01CB012C893D894E895F89821BDA
:1075A000930BA40BB50BB7FF07C0B095A0959095B2
:1075B00081959F4FAF4FBF4F4C0149815A81452B59
:1075C000F9F489E996E0FFD08EE496E0FCD086E1FC
:1075D00096E0F9D08889998969D18EE496E0F3D054
:1075E00088E196E0F0D0B401092C000C880B990BCF
:1075F0000E94BB4D42E05FD10E94D3180E94DD176C
:1076000085E090E0A985BA858D939C9345E050E094
:10761000B5018AA19BA10E942B19C5010E946D266C
:107620008AA19BA10E9487138AA19BA10E94891312
:10763000B1E02B163104A9F0E2E02E16310401F17D
:10764000232861F50E94D318C401990CAA0BBB0B27
:1076500080934A0790934B07A0934C07B0934D0734
:107660001DC00E94D318C401990CAA0BBB0B8093B8
:107670004E0790934F07A0935007B09351070EC049
:107680000E94D318C401990CAA0BBB0B809352071C
:1076900090935307A0935407B09355070E94D318B3
:1076A0000E943018A985BA851D921C9240E050E0D6
:1076B000B5018AA19BA10E942B1940E050E0B501C1
:1076C0008AA19BA10E9410190E94D318E981FA8116
:1076D000F0934507E093440789819A8111C08FEBAD
:1076E00096E071D0C5010E941726882309F496CD33
:1076F000B1E0BB8793CD0E9428268111BBCEB8CEC6
:10770000A3960FB6F894DEBF0FBECDBFDF91CF9129
:107710001F910F91FF90EF90DF90CF90BF90AF90AF
:107720009F908F907F906F905F904F903F902F90A1
:107730000895CF93DF93FC01E452FE4F40815181C5
:107740004115510559F1EC01C052DE4F28813981B4
:1077500088529E4F24173507C8F4FC01808191811F
:10776000009761F0FC01E20FF31F80818A3041F045
:107770008D3029F48CE993E026D002C080E064D0FB
:107780008881998101969983888308C040E050E000
:107790006EE973E00E94E60D19821882DF91CF91A5
:1077A0000895009769F0FC0101900020E9F73197F6
:1077B000AF01481B590BBC0188EA9BE00C942E0BCF
:1077C00080E090E00895EDCF8F929F92AF92BF92AC
:1077D0000F931F93CF93DF93CDB7DEB7A1970FB66B
:1077E000F894DEBF0FBECDBF19A2423008F44AE0C4
:1077F0008E010F5D1F4F842E912CA12CB12CA50161
:1078000094010E94134FE62FB901CA0101501109DA
:10781000EA3014F4E05D01C0E95CD801EC93232B5D
:10782000242B252B61F7C801BCDFA1960FB6F89475
:10783000DEBF0FBECDBFDF91CF911F910F91BF90E3
:10784000AF909F908F900895E091A80BF091A90BB5
:107850000190F081E02D682F88EA9BE01994CF9287
:10786000DF92EF92FF92CF93DF9397FF17C06B01E8
:107870007C018DE2E9DFEC0166277727CB016C19EB
:107880007D098E099F094AE09FDF8C0F9D1FDF91C4
:10789000CF91FF90EF90DF90CF9008954AE0DF9175
:1078A000CF91FF90EF90DF90CF908ECFBC01990FDA
:1078B000880B990BD4CF4F925F926F927F928F92E9
:1078C0009F92AF92BF92CF92DF92EF92FF926B01A5
:1078D0007C01B42E9B01AC010E944650882319F014
:1078E00086E397E027C026013701E89477F82FEF69
:1078F0003FEF4FE75FE7C301B2010E94465081119D
:107900000DC02FEF3FEF4FE75FE7C301B2010E94C9
:10791000B54D18161CF48AE397E00CC02FEF3FEF2B
:107920004FE75FE4C701B6010E94425018167CF48D
:107930008EE397E0FF90EF90DF90CF90BF90AF90F5
:107940009F908F907F906F905F904F902ACF2FEFF6
:107950003FEF4FE75FECC701B6010E94B54D87FDD1
:10796000E7CF20E030E0A901C701B6010E94B54D84
:1079700087FF08C08DE268DF4C01F7FAF094F7F852
:10798000F09402C0812C912CA12C60E070E080E08A
:107990009FE3AB1441F020E030E040E251E40E946C
:1079A000A94FA394F6CF9B01AC01C701B6010E9479
:1079B000454F2B013C010E9416506B017C010E9437
:1079C000B94D9B01AC01C301B2010E94444F2B0190
:1079D0003C014AE0C701B601F7DE7C01E80CF91C66
:1079E000BB2021F08EE230DFE80EF91EDB2CDD201B
:1079F00019F120E030E040E251E4C301B2010E94FD
:107A00001A4E2B013C010E9416504B01A12CB12CA7
:107A10004AE0C501B401D8DEE80EF91EC501B40183
:107A20000E94B94D9B01AC01C301B2010E94444FB9
:107A30002B013C01DA94DBCFC701FF90EF90DF9080
:107A4000CF90BF90AF909F908F907F906F905F90FE
:107A50004F900895789484B5826084BD84B5816028
:107A600084BD85B5826085BD85B5816085BD809109
:107A70006E00816080936E00109281008091810081
:107A80008260809381008091810081608093810079
:107A9000809180008160809380008091B10084603B
:107AA0008093B1008091B00081608093B00080919C
:107AB0009100826080939100809191008160809319
:107AC0009100809190008160809390008091A1004E
:107AD00082608093A1008091A10081608093A100C9
:107AE0008091A00081608093A0008091210182603C
:107AF00080932101809121018160809321018091F7
:107B0000200181608093200180917A0084608093BD
:107B10007A0080917A00826080937A0080917A0066
:107B2000816080937A0080917A00806880937A00E7
:107B30001092C10061E08AE10E949F0F61E08BE139
:107B40000E949F0F61E089E10E949F0F61E08FE03A
:107B50000E949F0F61E08EE10E949F0F61E08EE026
:107B60000E949F0F62E085E40E949F0F62E084E420
:107B70000E949F0F62E080E10E949F0F62E081E11E
:107B80000E949F0F61E080E20E949F0F61E081E20E
:107B90000E949F0F61E08FE10E949F0F62E083E4EB
:107BA0000E949F0F62E082E40E949F0F62E087E1E3
:107BB0000E949F0F62E088E10E949F0F61E083E2D4
:107BC0000E949F0F61E084E20E949F0F61E082E2C9
:107BD0000E949F0F62E081E40E949F0F62E080E4B8
:107BE0000E949F0F62E08DE10E949F0F62E08CE196
:107BF0000E949F0F61E088E20E949F0F61E089E28E
:107C00000E949F0F61E085E20E949F0F61E085E284
:107C10000E94AB0E61E08DE00E949F0F61E089E061
:107C20000E949F0F61E088E00E949F0F61E087E063
:107C30000E949F0F61E08AE00E949F0F61E08CE04C
:107C40000E949F0F62E08FE30E949F0F62E08BE330
:107C50000E949F0F61E084E00E949F0F61E085E039
:107C60000E949F0F61E086E00E949F0F61E08BE021
:107C70000E949F0F61E089E10E94AB0E61E08EE0FF
:107C80000E94AB0E61E08FE10E94AB0E61E082E2E8
:107C90000E94AB0EE091B80BF091B90B82E08083AB
:107CA000E091B40BF091B50B1082E091B60BF0911E
:107CB000B70BD0E1D0831092C00BE091BC0BF091D8
:107CC000BD0B86E08083E091BA0BF091BB0B808105
:107CD00080618083E091BA0BF091BB0B808188605A
:107CE0008083E091BA0BF091BB0B80818068808328
:107CF000E091BA0BF091BB0B80818F7D808364E6AD
:107D000070E080E090E00E94E60F0E9427170E943A
:107D1000C5130E94A0250E94611B0E941E10609343
:107D20007E0B70937F0B8093800B9093810B80E090
:107D300091E39093430780934207C1E0C0936F00A3
:107D4000D093810010928000C093DC0A80E092E022
:107D50009093DB0A8093DA0A9093870080938600E1
:107D600081E1809381001092810010928500109231
:107D700084008091DC0A8061809381000E941E1043
:107D800060937A0B70937B0B80937C0B90937D0BAD
:107D90000E941E106093820B7093830B8093840B60
:107DA0009093850B0E941E1060937E0B70937F0B47
:107DB0008093800B9093810B0E94453280915E07E7
:107DC00090915F07A0916007B09161070197A105AD
:107DD000B10581F40E9445328091A6079091A707D2
:107DE000A091A807B091A9070197A105B10511F4C9
:107DF0000C9400470E94453280915E0790915F0786
:107E0000A0916007B09161070197A105B10581F4C8
:107E10000E9445328091A2079091A307A091A407E8
:107E2000B091A5070197A105B10511F40C941F4766
:107E30000E94453280915E0790915F07A091600794
:107E4000B09161070197A105B10581F40E94453207
:107E500080919E0790919F07A091A007B091A107E4
:107E60000197A105B10511F40C943F4780E893E018
:107E7000AADCEFE72E2EE2E03E2EF5E7AF2EF2E091
:107E8000BF2E0E941E106093820B7093830B809311
:107E9000840B9093850B00917E0B10917F0B2091AA
:107EA000800B3091810B601771078207930748F4AC
:107EB00060937E0B70937F0B8093800B9093810B6C
:107EC0002CC0DC01CB01801B910BA20BB30B883EB5
:107ED0009340A105B10508F108511C4F2F4F3F4FAA
:107EE00000937E0B10937F0B2093800B3093810BBC
:107EF0000E94A025EC010E943312CE010C960E9434
:107F00003312CE0148960E943312CE0184960E940D
:107F10003312CE01C0960E94331288EA9BE00E9481
:107F20008E0B892B09F4BDC50E941E1060937A0B3D
:107F300070937B0B80937C0B90937D0B88EA9BE086
:107F40000E946C0B8093790B982F9F7D953479F06C
:107F50002091770B3091780BF901EB5BF44F808324
:107F60002F5F3F4F3093780B2093770B06C00E9412
:107F7000D31821E0DC011C962C938091770B909113
:107F8000780B8133910564F02AE02093790BFC0192
:107F9000EB5BF44F208301969093780B8093770BE3
:107FA0008091790B2091770B3091780B8A3039F4DE
:107FB000C9010197A2E1BBE0E5E4FBE004C0223384
:107FC0003105B4F76EC5AF0145545B4048175907FA
:107FD0001CF441914D93F7CFFC01EE5EF44F1082FB
:107FE000223031050CF459C581E193E0ECDB8EE4DD
:107FF00096E0E9DB8FE993E0E6DB82E19BE0E3DBFF
:108000008FE993E0E0DB8CE993E0DDDB8AE390E04D
:108010000E940E48EC011A821B821C821D821E8265
:108020001F82188619861A861B861C861D861E8648
:108030001F86188A198A1A8A1B8A1C8A1D8A1E8A18
:108040001F8A188E198E1A8E1B8E1C8E1D8E1E8EE8
:108050001F8E18A219A21AA21BA21CA21DA21EA248
:108060001FA218A619A61AA61BA61CA61DA61EA608
:108070001FA618AA19AA1AAA1BAA1CAA1DAA1EAAD8
:108080001FAA18AE19AE68E072E082E19BE00E9480
:108090003E498C01FC0180818654823008F027C162
:1080A00061EA73E0C8010E946251892B09F4D3C0D0
:1080B00064EA73E0C8010E946251892B09F4CBC0C5
:1080C00068EA73E0C8010E946251892B09F4C6C0B6
:1080D0006BEA73E0C8010E946251892B09F4BEC0AB
:1080E0006FEA73E0C8010E946251892B09F4B9C09C
:1080F00063EB73E0C8010E946251892B09F4B4C09C
:1081000067EB73E0C8010E946251892B09F4ACC08F
:108110006AEB73E0C8010E946251892B09F4A7C081
:108120006EEB73E0C8010E946251892B09F4A2C072
:1081300062EC73E0C8010E946251892B09F49DC072
:1081400066EC73E0C8010E946251892B09F498C063
:108150006AEC73E0C8010E946251892B09F493C054
:108160006EEC73E0C8010E946251892B09F48EC045
:1081700062ED73E0C8010E946251892B09F489C045
:1081800066ED73E0C8010E946251892B09F484C036
:108190006AED73E0C8010E946251892B09F47FC027
:1081A0006EED73E0C8010E946251892B09F47AC018
:1081B00062EE73E0C8010E946251892B09F475C018
:1081C00066EE73E0C8010E946251892B09F470C009
:1081D0006AEE73E0C8010E946251892B09F46BC0FA
:1081E0006EEE73E0C8010E946251892B09F466C0EB
:1081F00062EF73E0C8010E946251892B09F461C0EB
:1082000066EF73E0C8010E946251892B09F45CC0DB
:108210006AEF73E0C8010E946251892B09F457C0CC
:108220006EEF73E0C8010E946251892B09F452C0BD
:1082300062E074E0C8010E946251892B09F44DC0CC
:1082400066E074E0C8010E946251892B09F448C0BD
:108250008FEF9FEF47C080E090E044C081E090E066
:1082600041C08CE190E03EC08DE690E03BC08FE6DF
:1082700090E038C080E790E035C081E790E032C000
:1082800082E790E02FC083E790E02CC084E790E085
:1082900029C088E790E026C089E790E023C08AE7FC
:1082A00090E020C083E890E01DC084E890E01AC010
:1082B0008DE890E017C08EE890E014C08FE890E061
:1082C00011C080E990E00EC081EA90E00BC085EB20
:1082D00090E008C086EB90E005C087EB90E002C01C
:1082E00088EB90E09093010280930002BBC08FEF77
:1082F0009FEF9093010280930002B8C0D8018C9147
:10830000883539F4C8010196B6D76A837B838C839C
:108310009D83F8018081893539F4C8010196ABD776
:108320006E837F8388879987D8018C918A3539F449
:10833000C8010196A0D76A877B878C879D87F80143
:108340008081813449F4C801019695D70E9411506B
:108350006E877F87888B998BD8018C91823449F402
:10836000C801019688D70E9411506A8B7B8B8C8B39
:108370009D8BF8018081833449F4C80101967BD735
:108380000E9411506E8B7F8B888F998FD8018C91B2
:10839000833539F4C80101966ED76A8F7B8F8C8F35
:1083A0009D8FF8018081803549F4C801019663D71B
:1083B0000E9411506E8F7F8F88A399A3D8018C9152
:1083C000863549F4C801019656D70E9411506AA318
:1083D0007BA38CA39DA3F8018081873549F4C80154
:1083E000019649D70E9411506EA37FA388A799A731
:1083F000D8018C91853449F4C80101963CD70E947C
:1084000011506AA77BA78CA79DA7F80180818435AE
:1084100049F4C80101962FD70E9411506EA77FA77B
:1084200088AB99ABD8018C918D3449F4C801019681
:1084300022D70E9411506AAB7BAB8CAB9DABF8018D
:108440008081813549F4C801019615D70E941150E9
:108450006EAB7FAB88AF99AF6AE074E080E090E0EC
:108460000DD78C010115110509F048CF0E94D318D2
:10847000DC011C961C910E94453240906A07509086
:108480006B0760906C0770906D07CEA8DFA8E8AC12
:10849000F9AC0E94D318C0924607D0924707E092E9
:1084A0004807F092490780910002909101029924B7
:1084B00093948230910538F09C012F563109263073
:1084C000310508F0912C112371F08D36910559F08A
:1084D0009C01285731092330310528F0855B91092B
:1084E000039708F0D0C20E94453280915E079091B8
:1084F0005F07A0916007B09161070197A105B105E1
:1085000029F0992019F08DEF92E0BFC2209719F45D
:1085100089EF92E0BAC2E0900002F0900102BFEF52
:10852000EB16FB06A9F3E114F104B9F48091DD0A1E
:108530009091DE0A892B61F482E090E06FD521E111
:1085400032E0FC01318320839093DE0A8093DD0AC0
:108550000091DD0A1091DE0A6EC0FCE1EF16F10415
:10856000B9F48091DF0A9091E00A892B61F482E0EE
:1085700090E054D52BE132E0DC012D933C939093B5
:10858000E00A8093DF0A0091DF0A1091E00A53C0ED
:10859000BDE6EB16F104B9F48091E10A9091E20A8C
:1085A000892B61F482E090E039D525E232E0FC01CC
:1085B000318320839093E20A8093E10A0091E10ADB
:1085C0001091E20A53C0FFE6EF16F104B9F480916E
:1085D000E30A9091E40A892B61F482E090E01ED5D1
:1085E0002FE232E0DC012D933C939093E40A8093D8
:1085F000E30A0091E30A1091E40A53C000E010E09E
:10860000B0E7EB16F104B9F48091E50A9091E60A1F
:10861000892B61F482E090E001D529E332E0FC018E
:10862000318320839093E60A8093E50A0091E50A5E
:108630001091E60A6CC0F1E7EF16F104B9F48091ED
:10864000E70A9091E80A892B61F482E090E0E6D491
:1086500023E432E0DC012D933C939093E80A80936D
:10866000E70A0091E70A1091E80A6CC0B2E7EB163E
:10867000F104B9F48091E90A9091EA0A892B61F436
:1086800082E090E0CBD42DE432E0FC013183208302
:108690009093EA0A8093E90A0091E90A1091EA0AA4
:1086A0006AC0F3E7EF16F104B9F48091EB0A9091F8
:1086B000EC0A892B61F482E090E0B0D427E532E047
:1086C000DC012D933C939093EC0A8093EB0A00918C
:1086D000EB0A1091EC0A68C0B4E7EB16F104B9F4A8
:1086E0008091ED0A9091EE0A892B61F482E090E08E
:1086F00095D421E632E0FC01318320839093EE0A89
:108700008093ED0A0091ED0A1091EE0A68C0F8E737
:10871000EF16F104B9F48091EF0A9091F00A892BD9
:1087200061F482E090E07AD42BE632E0DC012D9314
:108730003C939093F00A8093EF0A0091EF0A109116
:10874000F00A68C0B9E7EB16F104A9F48091F10AC8
:108750009091F20A892B51F482E090E05FD4FC0101
:10876000B182A0829093F20A8093F10A0091F10AFB
:108770001091F20A6AC0FAE7EF16F104A9F48091A9
:10878000F30A9091F40A892B51F482E090E046D4E8
:10879000DC012D923C929093F40A8093F30A0091AD
:1087A000F30A1091F40A6CC0BDE8EB16F104B9F4B9
:1087B0008091F50A9091F60A892B61F482E090E0AD
:1087C0002DD429E832E0FC01318320839093F60A0E
:1087D0008093F50A0091F50A1091F60A6CC03EE804
:1087E000E316F104B9F48091F70A9091F80A892B05
:1087F00061F482E090E012D4E3E9F2E0DC01ED9371
:10880000FC939093F80A8093F70A0091F70A10916D
:10881000F80A6CC0FFE8EF16F104B9F48091F90A88
:108820009091FA0A892B61F482E090E0F7D3EDE9A8
:10883000F2E0DC01ED93FC939093FA0A8093F90A3D
:108840000091F90A1091FA0A6CC0F0E9EF16F104F0
:10885000B9F48091FB0A9091FC0A892B61F482E0C3
:1088600090E0DCD3E7EAF2E0DC01ED93FC93909337
:10887000FC0A8093FB0A0091FB0A1091FC0A6CC071
:10888000F1EAEF16F104B9F48091FD0A9091FE0A25
:10889000892B61F482E090E0C1D3E1EBF2E0DC01EE
:1088A000ED93FC939093FE0A8093FD0A0091FD0ADC
:1088B0001091FE0A6BC0F5EBEF16F104B9F480914C
:1088C000FF0A9091000B892B61F482E090E0A6D31F
:1088D000EBEBF2E0DC01ED93FC939093000B8093C3
:1088E000FF0A0091FF0A1091000B50C0F6EBEF1643
:1088F000F104B9F48091010B9091020B892B61F482
:1089000082E090E08BD3E5ECF2E0DC01ED93FC93A8
:108910009093020B8093010B0091010B1091020BBD
:1089200035C0F7EBEF16F104B9F48091030B909189
:10893000040B892B61F482E090E070D3EFECF2E05D
:10894000DC01ED93FC939093040B8093030B009157
:10895000030B1091040B1AC0F8EBEF16F104B1F4FD
:108960008091050B9091060B892B61F482E090E0D9
:1089700055D3E3EEF2E0DC01ED93FC939093060B0C
:108980008093050B0091050B1091060B0115110545
:1089900089F489EF92E00E94E33B0E94D3180E9481
:1089A000DD178EE094E00E94D13B8CE993E00E94B9
:1089B000D13B71C085EF92E00E94E33B0E94D31847
:1089C0000E94DD170E94D3181092450710924407A9
:1089D000E12CF12CFFEFEF1AFF0A21E0E216F1047F
:1089E00041F081EF92E00E94E33B0E94D3180E9485
:1089F000DD17D801ED91FC910480F581E02DBE01D9
:108A0000C80119950E94D318C0904407D09045071B
:108A10000E94D318FC018485E114F104D9F281117C
:108A20000AC0E414F5043CF4C114D10421F0F2E0CE
:108A3000CF16D10479F688EA9BE00E948E0B1816B7
:108A400019062CF488EA9BE00E946C0BF4CFCD2829
:108A500009F438C2992009F432C20E94453280914B
:108A6000660790916707A0916807B0916907019721
:108A7000A105B10509F023C20E94D31821E0DC0151
:108A80001C962C931CC281E093E00E94E33B0E9461
:108A9000D3180E94DD17CE0156D31092780B109296
:108AA000770B8091110B8111AAC00E94D318FC0191
:108AB0008485882309F4A3C00E942717EC01FC01D8
:108AC000E253FD4F108240960E946D26CE018657DC
:108AD0009F4F0E946D26CE018C5F9E4F0E946D2697
:108AE0000E946D357C018C01075C1F4FC1E0D0E016
:108AF0006801F8E3CF1AD108D6018C918823D9F008
:108B000084E294E00E94E33B88E294E00E94E33B2D
:108B1000CE010E94563C8CE993E00E94E33B60E06A
:108B20008C2F0E94AB0E40E050E0BE01C7010E94B6
:108B3000D732F6011082D8018C918823F9F084E2B3
:108B400094E00E94E33B8FE394E00E94E33BCE017C
:108B50000E94563C8CE993E00E94E33B61E08C2F3D
:108B60000E949F0F60E08C2F0E94AB0E41E050E00E
:108B7000BE01C7010E94D732F801108221960F5F13
:108B80001F4FC533D10509F0B3CF0E94C432809185
:108B9000DE0C90E09C01220F331F820F931FFC011B
:108BA000E35BF34F80818F7B80838091E10C90E0C9
:108BB0009C01220F331F820F931FFC01E35BF34FD5
:108BC00080818F7B80838091E40C90E09C01220F58
:108BD000331F820F931FFC01E35BF34F80818F7B78
:108BE00080838091E70C90E09C01220F331F820F5D
:108BF000931FFC01E35BF34F80818F7B80830E9496
:108C0000D318DC011C968C918093110BC0910F0B33
:108C1000D091100B0E944532FC0182819381C817CC
:108C2000D90799F00E944532DC0112968D919C91F2
:108C300013979093100B80930F0B0E9427170E949D
:108C4000C5130E94A0250E94611B0E941E10609304
:108C50000B0B70930C0B80930D0B90930E0B0091EC
:108C60007A0B10917B0B20917C0B30917D0B601760
:108C700071078207930708F4B6C0DC01CB01801BA3
:108C8000910BA20BB30B89389341A105B10508F4F0
:108C9000B4C00E94D318DC011C968C91882319F073
:108CA0008DE093E002C089E093E00E94E33B0E94E4
:108CB000D3180E94DD170E942717EC01FC01E7552D
:108CC000FD4F8081882341F0CE0182589E4F0E9443
:108CD00077366B017C0107C0FE01E25BFF4FC0806D
:108CE000D180E280F3800E94D318C0924A07D092CC
:108CF0004B07E0924C07F0924D07FE01E655FD4F01
:108D00008081882341F0CE0184569E4F0E947736A1
:108D10006B017C0107C0FE01E853FF4FC080D1808A
:108D2000E280F3800E94D318C0924E07D0924F0782
:108D3000E0925007F0925107FE01E555FD4F80810A
:108D4000882341F0CE0186549E4F0E9477366B01F6
:108D50007C0106C0CE5BDE4FC880D980EA80FB80F4
:108D60000E94D318C0925207D0925307E092540742
:108D7000F09255070E94D3180E9430180E942717BE
:108D80000E94BA190E94D3180E941A1B0E94D3187D
:108D90000E94EF170E94453280915E0790915F0715
:108DA000A0916007B09161070197A105B10541F05D
:108DB00085E093E00E94E33B0E94D3180E94DD17F8
:108DC0008091070B9091080BA091090BB0910A0BB1
:108DD0000196A11DB11D8093070B9093080BA093E2
:108DE000090BB0930A0B0E941E1060937A0B7093CC
:108DF0007B0B80937C0B90937D0B0E942B0C41C8C6
:108E000085E594E00E94E33B0E942717CF931F92D1
:108E10001F921F921F92812C912CA12CB12CC12C3E
:108E2000D12C760197018601B701A6010E94D502D7
:108E30000F900F900F900F900F900C94FA3E8DE6CC
:108E400094E00E94E33B0E9427171F9221E02F939A
:108E50001F921F921F92812C912CA12CB12CC12CFE
:108E6000D12C760197018601B701A6010E94D50297
:108E70000F900F900F900F900F900C94183F85E873
:108E800094E00E94E33B0E9427171F921F9221E06B
:108E90002F931F921F92812C912CA12CB12CC12CAD
:108EA000D12C760197018601B701A6010E94D50257
:108EB0000F900F900F900F900F900C94363F89EE0B
:108EC00092E002C08DEE92E00E94E33B0E94D31834
:108ED0000E94DD170E94D318109246071092470790
:108EE0001092480710924907D6CD8091450C909179
:108EF000460C29C11092AB0B1092AA0B88EE93E09E
:108F0000A0E0B0E08093AC0B9093AD0BA093AE0BC0
:108F1000B093AF0B8AE693E09093A90B8093A80BD4
:108F200085EC90E09093B50B8093B40B84EC90E0CB
:108F30009093B70B8093B60B80EC90E09093B90BB5
:108F40008093B80B81EC90E09093BB0B8093BA0BAD
:108F500082EC90E09093BD0B8093BC0B86EC90E08C
:108F60009093BF0B8093BE0B1092C10B1092C20B5B
:108F70001092C30B1092C40B82E090E04FD02CE70C
:108F800033E0FC013183208390934C0C80934B0C95
:108F90006EE973E085E49CE00E94100E8091DD0C88
:108FA000AEEDBCE09FEF48EB5BE0803378F48C9350
:108FB000282F30E0F901EE0FFF1F2E0F3F1FF901A0
:108FC000E35BF34F528341838F5F01C09C93139601
:108FD000FCE0AA3EBF0749F78093DD0C0895EF92AD
:108FE0000F931F93CF93DF93E80147FD02C034E056
:108FF00001C034E1E42F440FFF0BF7FF03C0F195EC
:10900000E195F109E32E022F2E2FAE01B3D1CE014F
:10901000DF91CF911F910F91EF900895CF93DF9340
:109020008230910510F482E090E0E091EE0CF09136
:10903000EF0C20E030E0C0E0D0E0309711F140814B
:10904000518148175907C0F04817590761F48281C8
:109050009381209719F09B838A832BC09093EF0C08
:109060008093EE0C26C02115310519F042175307E5
:1090700018F49A01BE01DF01EF010280F381E02DB7
:10908000DCCF2115310509F1281B390B24303105BE
:1090900090F412968D919C9113976115710521F0B2
:1090A000FB019383828304C09093EF0C8093EE0CBA
:1090B000FD01329644C0FD01E20FF31F81939193AD
:1090C000225031092D933C933AC02091EC0C309101
:1090D000ED0C232B41F420910402309105023093D2
:1090E000ED0C2093EC0C209102023091030221152B
:1090F000310541F42DB73EB7409106025091070269
:10910000241B350BE091EC0CF091ED0CE217F3070A
:10911000A0F42E1B3F0B2817390778F0AC014E5FE7
:109120005F4F2417350748F04E0F5F1F5093ED0C2B
:109130004093EC0C8193919302C0E0E0F0E0CF010A
:10914000DF91CF9108950F931F93CF93DF930097F3
:1091500009F48CC0FC013297138212820091EE0C4C
:109160001091EF0C0115110581F420813181820FDE
:10917000931F2091EC0C3091ED0C2817390779F5ED
:10918000F093ED0CE093EC0C71C0D80140E050E09E
:10919000AE17BF0750F412962D913C911397AD0175
:1091A0002115310509F1D901F3CF9D01DA0133838E
:1091B000228360817181860F971F8217930769F45C
:1091C000EC0128813981260F371F2E5F3F4F3183F5
:1091D00020838A819B8193838283452B29F4F0939A
:1091E000EF0CE093EE0C42C01396FC93EE931297B3
:1091F000ED01499159919E01240F351FE217F307A4
:1092000071F480819181840F951F029611969C9331
:109210008E938281938113969C938E931297E0E0B4
:10922000F0E0D80112968D919C911397009719F058
:10923000F8018C01F6CF8D919C9198012E5F3F4FE4
:10924000820F931F2091EC0C3091ED0C28173907F9
:1092500069F4309729F41092EF0C1092EE0C02C0D2
:10926000138212821093ED0C0093EC0CDF91CF91DE
:109270001F910F9108956627772709C24AEE5CE097
:1092800000C0FA01A191B081009719F41097E1F0A4
:10929000CD01DC01CD010D90002011F4C00113C0FF
:1092A000FB012191222319F02015D9F7F3CFFB01FF
:1092B0002191201519F41E92119606C02223C1F7A0
:1092C0000D900020A1F7D001FA01A193B083089579
:1092D000BB274A3031F4992322F4BDE29095819561
:1092E0009F4F30C0BB272A3051F4992342F4BDE28E
:1092F00090958095709561957F4F8F4F9F4F01C0DE
:10930000BB27FA01A62F6217710581059105330B62
:1093100030FB66F0AA27660F771F881F991FAA1FC8
:10932000A21710F0A21B63953850A9F7A05DAA33CD
:1093300008F0A95DA19336F7B111B1931082CA016B
:1093400004C4BB27FB015527AA27880F991FAA1F12
:10935000A41710F0A41B83955051B9F7A05DAA3350
:1093600008F0A95DA193009779F7B111B19311921B
:10937000CB01EBC34F925F926F927F929F92AF921D
:10938000BF92CF92DF92EF92FF920F931F93CF93F2
:10939000DF93CDB7DEB729970FB6F894DEBF0FBEC7
:1093A000CDBF6A01122FB02E2BE3201720F0FF242F
:1093B000F394F00E02C0BCE3FB2E0F2D27E0AE01AC
:1093C0004F5F5F4FCAD2AC018981982F997091305D
:1093D00031F0E1FC06C0E0FE06C090E205C09DE26F
:1093E00003C09BE201C090E0EE2DE07183FF3CC022
:1093F000911102C083E001C084E0811718F4212F8D
:10940000281B01C020E0E1110BC0F601822F30E2E1
:10941000882319F031938150FBCFC20ED11C20E07C
:10942000992329F0D6019C93F60131966F01C6016C
:109430000396E2FE0AC03EE4D6013C9341E4119655
:109440004C93119712963C9306C03EE6F60130838A
:1094500041E641833283FC01322F40E2332309F499
:1094600042C041933150FACF82FF44C0911102C0F3
:1094700083E001C084E0811718F4212F281B01C06C
:1094800020E0E1110BC0F601822F30E2882319F0B1
:1094900031938150FBCFC20ED11C20E0992329F0DB
:1094A000D6019C93F60131966F01C6010396E2FE48
:1094B0000BC039E4D6013C933EE411963C931197DE
:1094C00036E412963C9307C039E6F60130833EE657
:1094D000318336E63283FC01322F40E2332319F028
:1094E00041933150FBCFFC01E20FF11D10828EEF52
:1094F0009FEFB7C0F1E0911101C0F0E06F2F70E075
:109500001416150624F49A012F5F3F4F02C021E084
:1095100030E0260F371FBB2029F06B2D70E06F5F06
:109520007F4F02C060E070E0260F371F612F70E0B0
:10953000261737071CF4121B212F01C020E03E2DF7
:10954000387159F4D601322F60E2332319F06D934C
:109550003150FBCFC20ED11C20E0FF2331F0D601E9
:109560009C93B6016F5F7F4F6B01E1110BC0F60159
:10957000922F30E3992319F031939150FBCFC20E13
:10958000D11C20E09F2D940F3A81782F7071A72E67
:1095900084FF03C0313309F49150191624F4993033
:1095A00018F098E001C091E0E42F852F57FF02C02A
:1095B000E0E080E06E2F782FE0E0F0E0AEE29A2E5F
:1095C0003A01691A71082A01461A570A0B2D10E050
:1095D0001195019511096F3F8FEF780729F4D60196
:1095E0009C92C60101966C014617570784F06616D7
:1095F00077066CF47F01E40CF51CA1E0B0E0AC0F41
:10960000BD1FEA0EFB1ED7011196BC9002C090E36D
:10961000B92E615071093196C60101967C0160171F
:10962000710724F0D601BC926C01D5CF6417750781
:1096300041F4363320F4353321F4A11002C081E324
:10964000B82EF601B082F701822F90E2882319F03C
:1096500091938150FBCFF701E20FF11D108280E062
:1096600090E029960FB6F894DEBF0FBECDBFDF9114
:10967000CF911F910F91FF90EF90DF90CF90BF900F
:10968000AF909F907F906F905F904F9008956F92F2
:109690007F928F929F92AF92BF92CF92DF92EF9282
:1096A000FF920F931F93CF93DF93EC017B01611522
:1096B000710519F0DB018D939C938E010F5F1F4F95
:1096C0007880872D90E021D2892B11F0E801F5CF29
:1096D000BDE27B1205C00F5F1F4F7980C1E008C05B
:1096E000EBE27E1204C08E010E5F1F4F7980C0E056
:1096F0006801F1E0CF1AD10843E050E064EF72E076
:10970000C6010BD2892BE9F4680122E0C20ED11CFC
:1097100045E050E06FEE72E0C601FFD1892B21F4E5
:10972000680187E0C80ED11CE114F10419F0D701DB
:10973000CD92DC92C111F9C060E070E080E89FE753
:10974000FDC043E050E06CEE72E0C601E6D1892B2B
:1097500051F4E114F10409F4EDC00E5F1F4FF7015D
:1097600011830083E7C0680160E070E0CB0100E096
:1097700010E0F601D0EDD70DDA3050F52C2F226035
:10978000622E2C2F2870C2FF05C0211127C00F5F49
:109790001F4F24C0222311F001501109A5E0B0E0B1
:1097A0009B01AC0130D34B015C01880C991CAA1CB5
:1097B000BB1CC501B4016D0F711D811D911D683960
:1097C000A9E97A078A07A9E19A0740F0C66005C0AF
:1097D000DE3F51F4C3FD44C0C8606C2EBFEFCB1A0E
:1097E000DB0A7080C62DC5CF2D2F2F7D2531C1F509
:1097F00040814D3211F4C06106C04B3221F03196E8
:1098000021E030E006C03296D60111964C9122E05C
:1098100030E0A0EDA40FAA3018F0E21BF30B20C03B
:1098200040E050E04038BCE05B075CF49A01220F56
:10983000331F220F331F420F531F440F551F4A0F70
:10984000511D3196DF0111972C91A0EDA20FAA3086
:1098500048F3C4FF03C0519541955109040F151FEA
:10986000C1FF07C0E114F10421F03197D701ED9356
:10987000FC937FD1C370C33019F06B017C0106C02B
:109880006B017C01F7FAF094F7F8F09420E030E0F7
:10989000A901C701B60169D1882309F443C017FFA4
:1098A00006C0119501951109CBE0D3E002C0C3E2D7
:1098B000D3E05E01B8E1AB1AB1084601BE2DAF2D71
:1098C00090E2E92EF12C0E151F057CF0FE0125918A
:1098D000359145915491B4018B2F9A2FABD14B0107
:1098E000B82FA92F0E191F09EECF2497F594E794EE
:1098F000CA15DB0541F76401EB2EFA2E8E2D880F79
:109900008F2D881F8F3F41F020E030E0A901C70173
:10991000B6012BD1811106C082E290E09093F10C48
:109920008093F00CC701B60109C060E070E080E8E8
:109930009FEF04C060E070E080EC9FE7DF91CF9183
:109940001F910F91FF90EF90DF90CF90BF90AF905D
:109950009F908F907F906F900895283008F027E0B7
:109960003327DA01990F311D87FD9160009661055B
:10997000710539F432602E5F3D9330E32A95E1F7AB
:1099800008959F3F30F080387105610509F03C5F14
:109990003C5F3D93913008F08068911DDF93CF9339
:1099A0001F930F93FF92EF92192F987F9695E92FAF
:1099B00096959695E90FFF27EF57FC4F9927332788
:1099C000EE24FF24A701E70105900894079428F4EA
:1099D000360FE71EF81E491F511D660F771F881F9F
:1099E000991F0694A1F70590079428F4E70EF81E36
:1099F000491F561FC11D770F881F991F661F0694A8
:109A0000A1F70590079428F4F80E491F561FC71FA9
:109A1000D11D880F991F661F771F0694A1F7059027
:109A2000079420F4490F561FC71FD81F990F661FB0
:109A3000771F881F0694A9F784911095177041F03D
:109A4000D695C79557954795F794E7941A95C1F71A
:109A5000E7E2F3E068941590159135916591959141
:109A600005907FE27395E118F10A430B560BC90B81
:109A7000D009C0F7E10CF11E431F561FC91FD01DAE
:109A80007EF4703311F48A95E6CFE894015030F0FB
:109A9000080F0AF40027021708F4202F2395022F3D
:109AA0007A3328F079E37D932A95E9F710C07D9306
:109AB0002A9589F606949795679537951795179483
:109AC000E118F10A430B560BC90BD00998F0239506
:109AD0007E9173957A3308F070E37C932013B8F786
:109AE0007E9170617D9330F0839571E37D9370E397
:109AF0002A95E1F71124EF90FF900F911F91CF91DC
:109B0000DF91992787FD909508959111F6C08032D5
:109B100019F089508550D0F70895FB01DC014150C0
:109B2000504088F08D9181341CF08B350CF4805EB0
:109B3000659161341CF06B350CF4605E861B61111D
:109B400071F3990B0895881BFCCFDC01FC01672F92
:109B500071917723E1F7329704C07C916D93708304
:109B60006291AE17BF07C8F3089540D008F481E0B2
:109B70000895E89409C097FB3EF490958095709500
:109B800061957F4F8F4F9F4F9923A9F0F92F96E949
:109B9000BB279395F695879577956795B795F111BE
:109BA000F8CFFAF4BB0F11F460FF1BC06F5F7F4F5B
:109BB0008F4F9F4F16C0882311F096E911C077236D
:109BC00021F09EE8872F762F05C0662371F096E876
:109BD000862F70E060E02AF09A95660F771F881F45
:109BE000DAF7880F9695879597F90895990F0008E9
:109BF000550FAA0BE0E8FEEF16161706E807F9075F
:109C0000C0F012161306E407F50798F0621B730BF9
:109C1000840B950B39F40A2661F0232B242B252B7A
:109C200021F408950A2609F4A140A6958FEF811D1D
:109C3000811D08950BD07BC06CD028F071D018F036
:109C4000952309F05DC062C01124A5C081D0A0F3A6
:109C5000959FD1F3950F50E0551F629FF001729FC1
:109C6000BB27F00DB11D639FAA27F00DB11DAA1FE0
:109C7000649F6627B00DA11D661F829F2227B00D2D
:109C8000A11D621F739FB00DA11D621F839FA00DB8
:109C9000611D221F749F3327A00D611D231F849F08
:109CA000600D211D822F762F6A2F11249F5750405F
:109CB0008AF0E1F088234AF0EE0FFF1FBB1F661FFA
:109CC000771F881F91505040A9F79E3F510570F0B3
:109CD00017C061C05F3FECF3983EDCF38695779543
:109CE0006795B795F795E7959F5FC1F7FE2B880FAE
:109CF000911D9695879597F9089599278827089536
:109D000097F99F6780E870E060E008959FEF80EC2E
:109D1000089500240A9416161706180609060895D1
:109D200000240A9412161306140605060895092E37
:109D30000394000C11F4882352F0BB0F40F4BF2BA6
:109D400011F460FF04C06F5F7F4F8F4F9F4F0895E6
:109D500057FD9058440F551F59F05F3F71F04795DC
:109D6000880F97FB991F61F09F3F79F087950895C1
:109D7000121613061406551FF2CF4695F1DF08C0E0
:109D8000161617061806991FF1CF869571056105FD
:109D900008940895E894BB2766277727CB0197F9A5
:109DA0000895F999FECF92BD81BDF89A992780B5A3
:109DB0000895262FF999FECF1FBA92BD81BD20BD0F
:109DC0000FB6F894FA9AF99A0FBE01960895052EE7
:109DD00097FB16F400940FD057FD05D024D007FC54
:109DE00002D046F408C050954095309521953F4FDC
:109DF0004F4F5F4F089590958095709561957F4F77
:109E00008F4F9F4F089531D0A59F900DB49F900D17
:109E1000A49F800D911D11240895B7FFF4CFF3DFA7
:109E2000821B930B0895A1E21A2EAA1BBB1BFD01F6
:109E30000DC0AA1FBB1FEE1FFF1FA217B307E40729
:109E4000F50720F0A21BB30BE40BF50B661F771F81
:109E5000881F991F1A9469F7609570958095909561
:109E60009B01AC01BD01CF010895A29FB001B39F3A
:109E7000C001A39F700D811D1124911DB29F700D13
:109E8000811D1124911D08955058BB27AA270ED07B
:109E90004ECF3FDF30F044DF20F031F49F3F11F42C
:109EA0001EF434CF0EF4E095E7FB2ACFE92F50DF04
:109EB00080F3BA17620773078407950718F071F4E7
:109EC0009EF568CF0EF4E0950B2EBA2FA02D0B0156
:109ED000B90190010C01CA01A0011124FF27591BEF
:109EE00099F0593F50F4503E68F11A16F040A22FF5
:109EF000232F342F4427585FF3CF46953795279566
:109F0000A795F0405395C9F77EF41F16BA0B620B64
:109F1000730B840BBAF09150A1F0FF0FBB1F661FAB
:109F2000771F881FC2F70EC0BA0F621F731F841FEE
:109F300048F4879577956795B795F7959E3F08F014
:109F4000B3CF9395880F08F09927EE0F97958795D3
:109F500008950CD0ECCEE4DE40F0DBDE30F021F4EE
:109F60005F3F19F0CDCE511116CFD0CEF1DE98F370
:109F70009923C9F35523B1F3951B550BBB27AA278A
:109F800062177307840738F09F5F5F4F220F331FFC
:109F9000441FAA1FA9F333D00E2E3AF0E0E830D0C8
:109FA00091505040E695001CCAF729D0FE2F27D0CB
:109FB000660F771F881FBB1F261737074807AB0799
:109FC000B0E809F0BB0B802DBF01FF2793585F4F0E
:109FD0002AF09E3F510568F093CEDDCE5F3FECF353
:109FE000983EDCF3869577956795B795F7959F5FD3
:109FF000C9F7880F911D9695879597F90895E1E027
:10A00000660F771F881FBB1F621773078407BA0785
:10A0100020F0621B730B840BBA0BEE1F88F7E095E0
:10A02000089504D06894B111B6CE089599DE88F0F1
:10A030009F5790F0B92F9927B751A0F0D1F0660F34
:10A04000771F881F991F1AF0BA95C9F712C0B1304F
:10A0500081F0A0DEB1E008959DCE672F782F88278C
:10A06000B85F39F0B93FCCF3869577956795B3958E
:10A07000D9F73EF490958095709561957F4F8F4FFD
:10A080009F4F0895B3DD08F48FEF0895AFDD880B7F
:10A09000990B0895DB018F939F93B5DEBF91AF912C
:10A0A000A29F800D911DA39F900DB29F900D112432
:10A0B0000895991B79E004C0991F961708F0961B24
:10A0C000881F7A95C9F780950895EE0FFF1F881FA6
:10A0D0008BBF0790F691E02D19946F927F928F922B
:10A0E0009F92AF92BF92CF92DF92EF92FF920F9327
:10A0F0001F93CF93DF93EC01009789F4CB01DF919D
:10A10000CF911F910F91FF90EF90DF90CF90BF9074
:10A11000AF909F908F907F906F900C940E48FC01B1
:10A12000E60FF71F9C0122503109E217F30708F4EC
:10A13000ABC0D9010D911C91119706171707B0F00C
:10A140000530110508F49EC0C801049786179707CB
:10A1500008F498C002501109061B170B01931193C4
:10A160006D937C93CF010E94A3488CC05B01A01A21
:10A17000B10A4C01800E911EA091EE0CB091EF0C33
:10A1800040E050E0E12CF12C109709F44AC0A815EA
:10A19000B905D1F56D907C901197630182E0C80EEE
:10A1A000D11CCA14DB0480F1A3014A195B096A01BE
:10A1B00082E0C80ED11C1296BC9012971396AC91F7
:10A1C000B5E0CB16D10440F0B282A3835183408323
:10A1D000D9016D937C930AC00E5F1F4FC301800F9E
:10A1E000911FF90191838083EB2DFA2FE114F10483
:10A1F00031F0D7011396FC93EE93129743C0F0937E
:10A20000EF0CE093EE0C3EC08D919C911197481796
:10A21000590708F4AC017D0112960D90BC91A02D58
:10A22000B3CF8091EC0C9091ED0C88159905E1F479
:10A2300046175707C8F480910202909103020097D5
:10A2400041F48DB79EB74091060250910702841BDE
:10A25000950BE817F907C0F4F093ED0CE093EC0CC4
:10A26000F901718360830EC0CB010E940E487C010E
:10A27000009751F0A801BE011CD0CE010E94A34856
:10A28000C70104C0CE0102C080E090E0DF91CF9111
:10A290001F910F91FF90EF90DF90CF90BF90AF9004
:10A2A0009F908F907F906F90089581E090E0F89458
:10A2B00019C0FB01DC0102C001900D9241505040D9
:10A2C000D8F70895FB01DC018D91019080190110F0
:10A2D000D9F3990B0895FB01DC0101900D92002048
:10A2E000E1F7089512E0C2EAD2E000E005C0802F55
:10A2F000FE01EBDE2196011DC33AD10780E008077D
:06A30000B1F7F894FFCF55
:10A30600FFFF0000F20C8000200A0D000000000094
:10A31600009517C1134017000000009617C3136F6E
:10A326001A00000000C3366434663500000000CF12
:10A3360025F924452500000000CA12E20C440D0050
:10A34600000000C33295308331000000000E3656FF
:10A3560034683400000000C2366234A034000000C5
:10A36600003212E00C0B0D00000000BF365C3436E4
:10A3760035000000006A2BFD249125000000000F27
:10A38600365834D83400000000C4366634F135003F
:10A3960000000010365A34C73500000000C1366090
:10A3A60034DB35000000000D3652348C35000000D9
:10A3B60000CD25F524FF2400000000C13291304372
:10A3C6003300000000D025FB24762500000000C0E5
:10A3D600365E34593500000000CE25F724DA240015
:10A3E600000000C232933097305230330052303280
:10A3F600005230370052303100523039005238386E
:10A406000052383700523838005230300052383750
:10A41600005230380052313300523132005231315D
:10A42600005237330052373200523731005231373B
:10A4360000523136005231350001000000010000A3
:10A4460000010000005238350052383400523035D1
:10A456000052303600362E342E322E460000523050
:10A4660034005238370000000000C40B2E0B5D0B81
:10A476000A0C8E0B6C0B800B000000000C3654345B
:10A486005239392041524455494E4F205354415276
:10A4960054555020434F4D504C4554450D0A002A03
:10A4A6000047300047303000473100473031004721
:10A4B60032380046303900463900463131004631DF
:10A4C60032004631330046313400463135004631DC
:10A4D60036004632300046323100463232004633CC
:10A4E60031004633320046343100463432004634B9
:10A4F600330046343400463631004638310046389B
:10A5060032004638330046383400200A0D005239EE
:10A51600392068616E646C6572203D3D204E554C55
:10A526004C0D0A00523939002072657365747469DE
:10A536006E67206469676974616C2070696E0020BB
:10A54600726573657474696E6720616E616C6F679E
:10A556002070696E0052393920484F4D45205A20E7
:10A566004F4E20535441525455500D0A005239391A
:10A5760020484F4D452059204F4E205354415254A8
:10A5860055500D0A0052393920484F4D4520582064
:10A596004F4E20535441525455500D0A00523939EA
:10A5A60020656D657267656E63792073746F700DD3
:10A5B6000A00523939206572726F720D0A005238DC
:10A5C60032005239392073746F707065640D0A0059
:10A5D600523939206572726F72200020646561639A
:10A5E600746976617465206D6F746F72205820648B
:10A5F600756520746F206D69737365642073746567
:10A606007073002064656163746976617465206D9A
:10A616006F746F7220592064756520746F206D69A0
:10A626007373656420737465707300206465616379
:10A63600746976617465206D6F746F72205A206438
:10A64600756520746F206D69737365642073746516
:10A656007073005239392074696D656F75742058AE
:10A6660020617869730D0A005239392074696D6565
:10A676006F7574205920617869730D0A0052393953
:10A686002074696D656F7574205A20617869730D41
:10A696000A0020510052383100205841002058420B
:10A6A600002059410020594200205A4100205A42B8
:10A6B6000020737461200020637572200020656E8F
:10A6C6006420002068616C662000206C656E2000A6
:10A6D600206D696E2000206D617820002073706403
:10A6E60020005239392057696C6C207A65726F20C8
:10A6F60058005239392057696C6C207A65726F2080
:10A7060059005239392057696C6C207A65726F206E
:10A716005A005232310050005600523939204572E3
:10A72600726F723A20696E76616C6964207061722C
:10A73600616D657465722069640D0A0052343100DA
:10A74600686F6D650D0A00523230005238332000B2
:10A756005239392043616C6962726174696F6E2087
:10A766006572726F723A20696E76616C69642061F7
:10A776007869732073656C65637465640D0A0020DF
:10A786006178697320002061742073746172746942
:10A796006E6720706F696E740052323300206361F9
:10A7A6006C6962726174696E67206C656E67746845
:10A7B60000207374657020636F756E743A200052C2
:10A7C6003939206D6F76656D656E7420646F6E65C0
:10A7D6000D0A0020617420656E6420706F696E74C6
:10A7E600005239392043616C6962726174696F6E17
:10A7F600206572726F723A20656E642073746F7092
:10A8060020616374697665206265666F7265207380
:10A81600746172740D0A00206D6F766520746F2066
:10A82600737461727420666F722063616C69627200
:10A836006174696F6E006E616E00696E66006F7698
:02A846006600AA
:00000001FF
